:020000040800F2
:100000003811002001010008033800089928000871
:1000100001380008350F0008D16300080000000017
:10002000000000000000000000000000054900087A
:10003000671A0008000000006D3D0008054C00082C
:100040001B010008613B00081B0100081B010008A0
:100050001B0100081B0100081B0100081B01000810
:100060001B0100081B0100081B0100081B01000800
:100070001B0100081B010008211500081B010008D6
:100080001B0100081B0100083D0700081B010008B8
:100090001B0100081B0100081B0100081B010008D0
:1000A000754C0008614D00081B0100081B01000889
:1000B000654D000851500008AD5200081B010008B2
:1000C0001B0100081B0100081B0100081B010008A0
:1000D0001B010008C95E00081B0100081B01000885
:1000E0001B0100081B0100081B010008DFF80CD0F1
:1000F00000F0E6FA0048004741750008381100207A
:100100000648804706480047FEE7FEE7FEE7FEE7B1
:10011000FEE7FEE7FEE7FEE7FEE7FEE7254C000808
:10012000ED0000082DE9F0410024061B254671F181
:10013000000605DA01240027D0EB070067EB010178
:10014000161E73F1000605DA0027D2EB070201251F
:1001500067EB030300F0D0F986460E4617469C462F
:10016000AC4204D00025D0EB050E65EB010624B1AE
:100170000020D2EB000760EB030C704631463A4694
:100180006346BDE8F08140EA01039B0703D009E024
:1001900008C9121F08C0042AFAD203E011F8013B73
:1001A00000F8013B521EF9D2704780EA010210B5F7
:1001B00002F00043400022D04A001FD0010E01EBA4
:1001C0001261C0F35600C2F3560240F4000042F43C
:1001D0000002A0FB022000047F39140400D0401C60
:1001E00050EA124001D44000491EC2B20C0604EB92
:1001F000D010401C4008802A02D003E0002010BD2F
:1002000020F00100002900DA0020184310BD2DE97C
:10021000FE4F81EA030404F0004421F00041009401
:100220004FF0000B23F0004350EA01045ED052EA85
:1002300003045BD0C3F30A54C1F30A552C44A4F25F
:10024000F3340194A0FB0254C1F3130141F4801173
:10025000C3F3130343F4801301FB024400FB034E7A
:10026000840A970A44EA815447EA8357A4FB076843
:1002700002958D0A05FB07854FEA932C04FB0C546D
:100280002705029D4FEA065847EA1637B5EB0805E1
:100290006EEB070C870E920E47EA811742EA831233
:1002A000A7FB0201B6EB0B0164EB00042B0D43EA44
:1002B0000C335E1844EB1C50DA465146E7FB020152
:1002C000C5F313044FEA0B3343EA14534FEA0432E5
:1002D000019C43EA0603A4F10C040294009CCDE9BE
:1002E00000B400F09FF903B0BDE8F08F0020014694
:1002F000F9E72DE9F04D81EA030404F0004B21F009
:10030000004514464FF0000A23F0004150EA050270
:1003100020D054EA01021DD0C5F30A570246C5F3A6
:100320001303C1F31300C1F30A5640F4801543F4DC
:100330008013A7EB0608101BD64608F2FD3873EBB6
:10034000050002D308F1010801E092185B41B8F101
:10035000000F03DA00200146BDE8F08D00204FF4C5
:100360008011064684460EE0171B73EB050705D384
:10037000121B63EB050306434CEA010C49084FEAE4
:10038000300092185B4150EA0107EDD152EA0300B8
:1003900012D082EA040083EA0501084305D0101B4D
:1003A000AB4106D20122002306E000224FF00043B9
:1003B00002E06FF0010253101AEB06004CEB0851FB
:1003C00010EB0A0041EB0B01BDE8F04D00F01BB94A
:1003D00070B521F0004303430CD0C1F30A5500244B
:1003E000D5EB040564EB0403D617AD1AB34102DB69
:1003F0000020014670BD201841EB025170BDC10FB5
:1004000080EAE0700844CA079623002100F0CDB8C6
:1004100096230022114600F0C8B80EB5C10F80EA3D
:10042000E0700844CA07002140F233438DE80E0013
:100430000A460B4600F0F6F803B000BD0EB540F2D8
:10044000334102910021CDE900110A460B4600F02C
:10045000E9F803B000BD00F0004220F00040C10DFB
:10046000C0F3160040F400007F2901DA0020704735
:10047000962903DCC1F19601C84001E09639884015
:10048000002AF4D04042704770B5C1F30A5201F01F
:1004900000450024C1F3130140F2FF3341F4801101
:1004A0009A4201DA002070BD40F233439A42A2F230
:1004B000334203DC524200F05FF800E090402C43EE
:1004C000F1D0404270BDC1F30A5210B5C1F313011F
:1004D00040F2FF3341F480119A4201DA002010BD4E
:1004E00040F233439A42A2F2334203DC524200F01C
:1004F00043F810BD904010BD2DE9F05F0546002087
:1005000092469B4688460646814640241BE0284684
:1005100041464746224600F02FF853465A46C01A35
:10052000914110D311461846224600F016F82D1AB4
:1005300067EB01084F4622460120002100F00DF82C
:1005400017EB00094E41201EA4F10104DFDC4846F0
:1005500031462A464346BDE8F09F202A04DB203A74
:1005600000FA02F1002070479140C2F1200320FA06
:1005700003F3194390407047202A04DB203A21FA04
:1005800002F00021704721FA02F3D040C2F12002AC
:1005900091400843194670470029A8BF7047401C86
:1005A000490008BF20F00100704710B4B0FA80FC89
:1005B00000FA0CF050EA010404BF10BC704749B1C6
:1005C000CCF1200421FA04F411FA0CF118BF012136
:1005D00021430843A3EB0C01CB1D4FEA00614FEA16
:1005E000102042BF002010BC704700EBC3501044E5
:1005F0000029A4BF10BC7047401C490008BF20F070
:10060000010010BC704710B5141E73F1000408DA25
:10061000401C41F1000192185B411A4301D120F0C6
:10062000010010BD2DE9F04D92469B4611B1B1FA83
:1006300081F202E0B0FA80F220329046FFF78DFF9F
:1006400004460F4640EA0A0041EA0B0153465A4667
:10065000084313D0114653EA010019D0C8F14002F3
:100660005046FFF789FF05460E465046594642461A
:10067000FFF773FF084305D0012004E02046394608
:10068000BDE8F08D0020054346EAE0762C43374371
:100690000A986305E40AA0EB08000022FD0A44EA78
:1006A00047540A3002D500200146E9E70105101938
:1006B0006941DDE9084500196941BDE8F04DA2E74F
:1006C000064C074D06E0E06840F0010394E807009F
:1006D00098471034AC42F6D3FFF70CFD2C98000875
:1006E0004C98000870B58C1810F8015B15F00703E2
:1006F00001D110F8013B2A1106D110F8012B03E0BB
:1007000010F8016B01F8016B5B1EF9D12B0705D4C2
:100710000023521E0DD401F8013BFAE710F8013B0B
:10072000CB1A921C03E013F8015B01F8015B521E27
:10073000F9D5A142D8D3002070BD000070B54C4C53
:100740004FF490652946204600F015FA002864D041
:100750002946204600F0A2F846490888401C088037
:100760000121204600F0E6FA434942F21072B1F846
:100770005800904202D2401CA1F8580007F0C4F87B
:100780003E4DB5F91410B5F9120005F085FF3C4C4B
:10079000A5F856002080A16820468847A088A5F8C3
:1007A000580003F097F807F0ABF9364E364C307826
:1007B000082833D045F6AC30606042F6EF60A060A8
:1007C00042F2C400E0603148008A2080208E6080C0
:1007D000A16B2D488847208E69882D4C08444FF620
:1007E000FF7101EA80006887207A4FF0000540071A
:1007F0001DD501F0C7FA274949F6A24008802648CE
:1008000040F21A62C188491C89B2C180914204D366
:10081000A16821F00401A160C58070BD41F2130000
:1008200060604FF48060A06040F61B50CAE73078EB
:100830000A2818D2DFE800F0170613050A050D177D
:100840001113EAE7BDE8704006F0D0B808F028F9C7
:1008500005E0BDE8704002F087BD06F04DFCBDE844
:10086000704007F0A5BA00F0FDFB84F8B65070BDEB
:10087000002401402C0700204801002064000020D3
:100880004C07002023070020E40000200002002085
:10089000AC020020442C01406C0900206FEA1121B9
:1008A000016070470029816802D041F0010101E038
:1008B00021F00101816070470029816802D041F474
:1008C000807101E021F48071816070472DE9F04171
:1008D000824E92B0304600F00BF90BA800F039FAC6
:1008E00001214FF4C06003F0D5FA00248DF83140A7
:1008F0004FF46020CDE90D044FF4A0204FF009081B
:100900000B9001278DF83C808DF830700BA9304694
:1009100000F080F9724D8DF831408DF830708DF80F
:100920003C700BA9284600F075F901231A460F21E7
:10093000304600F0C0F9022201231146304600F093
:10094000BAF9012303220021304600F0B4F9012353
:1009500004221946304600F0AEF9012305220B218E
:10096000304600F0A8F9012306220421304600F0A9
:10097000A2F9012307220821304600F09CF9012347
:1009800008220321304600F096F9012309220A21AA
:10099000304600F090F90121304600F084F9012141
:1009A000284600F080F901231A460521304600F060
:1009B00055F901231A460621284600F04FF9002177
:1009C000304600F0CBF84FF4E041284600F0C6F87E
:1009D0000121304600F0B8F80121284600F0B4F8B3
:1009E0000121304600F0A6F80121284600F0A2F8C7
:1009F0000121304600F09EF90121284600F09AF9C5
:100A000040F61451374804F028FF12208DF84000BA
:100A100002208DF841008DF842408DF8437010A8F7
:100A200002F01CFF01224FF49061304600F0E8F81C
:100A300001213046FFF740FF01213046FFF732FF2A
:100A400001212846FFF72EFF304600F06EF93046B0
:100A500000F09FF80028FAD1304600F075F93046D2
:100A600000F082F80028FAD1284600F05EF9284606
:100A700000F08FF80028FAD1284600F065F92846E2
:100A800000F072F80028FAD10121084603F0DEF9DF
:100A9000154D284600F080FD684600F028FE0F48FE
:100AA00001A94C300090114881E811018020CDE966
:100AB00004404000069080000790202008904FF4EA
:100AC0004050CDE909046946284600F0F3FD0121B4
:100AD000284600F055FD12B0BDE8F0810024014029
:100AE00000280140002C014008000240BC02002008
:100AF0000D4910B5884202D1012144150AE00B4985
:100B0000884202D10121041504E0094988420AD132
:100B10000121CC03204603F0C9F92046BDE810406E
:100B2000002103F0C3B910BD00240140002801409A
:100B3000003C01400029816802D041F4801101E0AD
:100B400021F48011816070470029816802D041F44E
:100B5000004101E021F4004181607047826822F485
:100B6000E0420A43826070470146002089684907D5
:100B700000D50120704710B50246002054680B0ACA
:100B8000C9B20C401168194202D0002C00D00120DB
:100B900010BD014600208968090700D50120704773
:100BA00038B501211C2003F075F9FF20ADF80000D5
:100BB00000248DF8034003258DF8025069460D4846
:100BC00001F0DAFA0120ADF800008DF803408DF84D
:100BD00002506946084801F0CFFA2320ADF8000022
:100BE0008DF803408DF802506946044801F0C4FABC
:100BF00038BD000000080140000C01400010014019
:100C0000002A4268C9B201D00A4300E08A43426028
:100C10007047000010B542680E4B0C791A400B6803
:100C200042EA04221343436083680B4A1340D1E92C
:100C3000024222434C7943EA44031A438260C26A67
:100C4000097C22F47002491EC9B242EA0151C16214
:100C500010BD0000FFFEF0FFFDF7F1FF70B50724A7
:100C600009290AD9C568A1F10A0606EB4606B4406F
:100C7000A543B3401D43C56007E0056901EB41068C
:100C8000B440A543B3401D430561836BC3F30154D6
:100C9000121B921C02EB82041F22A2409343A1402C
:100CA0000B43836370BD826B491E22F4401242EAFB
:100CB00001518163704770B5072409290AD9C568B5
:100CC000A1F10A0606EB4606B440A543B3401D4316
:100CD000C56007E0056901EB4106B440A543B34098
:100CE0001D4305611F23072A09D2446B521E02EBE4
:100CF000820293409C4391400C43446370BD0D2A93
:100D000009D2046BD21F02EB820293409C439140B4
:100D10000C43046370BDC46A0D3A02EB8202934037
:100D20009C4391400C43C46270BD816841F008014E
:100D3000816070470029816802D041F4A00101E080
:100D400021F4A00181607047816841F00401816055
:100D5000704700210160017141718160C160012112
:100D60000174704770B51E4C214694F83800B1F8F4
:100D7000425006281ED9B4F84A10B4F84C00A1EB32
:100D8000000202F10902122A04D8FFF757FB0022E1
:100D9000144B0AE0884204D2FFF750FB0022124BAA
:100DA00003E0FFF74BFB0022104BFFF730FAFFF791
:100DB0008AFB09E005D12846FFF740FB0C4A0D4BA2
:100DC000F3E70D4951F82000C5EB45116063B0EB26
:100DD000410F03D9C5EB45104000606370BD0000B2
:100DE000580400200000344000003340000035402B
:100DF0006766666666E64B40DC8E000810B50C4CF4
:100E00002078400713D5FFF7ADFF0A49A08E088070
:100E100008483038018821F010010180001F018846
:100E200041F010010180207820F00400207010BDF6
:100E30005804002040040040F0B4184816494FF40C
:100E40009677436C08468A68046815485FEAC25C76
:100E500042F00806007822F008054FEA047415D520
:100E6000002C08DB120714D408B1082811D1BB42AA
:100E70000FDA8E6007E012070BD508B1082808D1F9
:100E8000BB4206DA8D60F0BC05F038BF002CF2DA08
:100E9000E8E7F0BC70470000AC02002048010020E9
:100EA0002307002070B506464089204B204C4FF4A4
:100EB0008071002580B362887AB1012A0CD1E18863
:100EC000491C89B2E1803289914205D36580E58071
:100ED000FF2801D0401E708170BD7088228890422A
:100EE00001D9012200E00022184601F0CEF97088F5
:100EF000B18801442088401C80B220808142EBD818
:100F00002580A088401C80B2A080F1888842E3D36D
:100F100001206080A58070BDFFE70022184601F027
:100F2000B4F9A580E58025806580F4E7000C0140D8
:100F3000C8050020FEE70000FCB505464FF6FF7629
:100F400000200C46ADF8006048F205078DF804005B
:100F500020E000BF15F8010B8DF8040001A9084638
:100F600002F0BFF8BDF800009DF8041080EA0120EF
:100F7000ADF800005FF00000BDF800100A0402D5D3
:100F800087EA410101E006EA4101401CADF800108A
:100F90000828F1DB641EDDD26946084602F08BF8B2
:100FA000BDF80000FCBD00000246002004E000BFC8
:100FB00012F8013B1844C0B2491EF9D27047000034
:100FC00070B5144A85B01088002413490194009428
:100FD000039420460494138807E00D8B009E35444B
:100FE0000095CD8B019E3544019515889D42F4D026
:100FF000401CC0B28028EED30098411107484180C0
:10100000848001984111064881830183818205B063
:1010100070BD00002C070020AC020020E20500207B
:10102000D004002030B50E4902880A800C4A43885B
:10103000083A13800B1F808818802024151F2C80ED
:101040000020401C80B27328FBD341F211100880AD
:1010500044F64800108047F2480018802C8030BDCC
:10106000202C0140114944F648000880091D46F62D
:1010700048000880091D41F2111008800B48001F2C
:10108000018841F02001018009480021A0F8641086
:10109000A0F86210A0F86010A0F85E10A0F85C1034
:1010A000A0F85A100348418181827047182C0140F2
:1010B000AC020020640000202DE9F0474F4B50485F
:1010C0000021DA7A0578802A25F001047ED34D4E7E
:1010D00002F01F021B6856F82220DFF82C81134211
:1010E000D8F8002002D042F0200201E022F02002D5
:1010F000484EC8F80020DFF814A1B6F90470424E3B
:101100009AF80030DFF8089196F84660022B62D119
:10111000B8F80830C3F3C00CC3F300239C455AD081
:10112000394B2C3B93F802C0BCF1000F06D0BCF148
:10113000010F0DD0BCF1020F52D124E011054FD5A3
:1011400091064DD40121997025F00401017047E00A
:10115000140545D4940643D56C0741D44488B4BBE8
:10116000DFF8B4C0BCF8504024B24480002C08DD45
:1011700045F00501017002219970BCF8441001820C
:101180002EE099702CE0C5880DB9002F12DC057B8C
:10119000B5420FD1214DAD895FEA457C0AD45FEAA3
:1011A000857C07D45FEA427C04D55FEA826C01D576
:1011B000ED0715D004704180A9F80010418141610C
:1011C00081610182997088F80F1001E011E007E059
:1011D0008AF8001004E004704180A9F800104181F1
:1011E000C7800673500960F3CB22C8F80020BDE821
:1011F000F087047041804181F9E70000E805002094
:10120000500900203C930008AC0200202307002076
:1012100024010020E205002048010020600A00208F
:101220002DE9F04796B000240C940D940E940F9481
:1012300072B69048816941F400718161816941F41D
:10124000806181614FF4004002F0F6FD8A4D00217B
:101250002846FFF731FB00212846FFF723FB874E86
:1012600000213046FFF71EFB854F0021384600F075
:1012700087F901204FF47041401C8842FCD3284676
:10128000FFF736FCB1463046FFF732FC384600F037
:1012900083F94FF46020CDE912048DF84540012018
:1012A0004FF004088DF8440010948DF8508010A978
:1012B0002846FFF7AFFC01231A4605212846FFF711
:1012C000FAFC0123022206212846FFF7F4FC012341
:1012D000032207212846FFF7EEFC012304220F21F9
:1012E0002846FFF7E8FC384600F056F9684600F05B
:1012F000FEF96148634E4C300090CDF80C80CDE98A
:1013000001648020CDE904404000069080000790F1
:10131000202008904FF44050CDE909046946384632
:1013200000F0C8F901212846FFF7C6FA0121384626
:1013300000F026F901212846FFF7B4FA47F23051B0
:1013400015941598401C15908842FAD3012128461F
:10135000FFF7F0FCADF82C40A04640F2DC5A4FF409
:10136000007420E05046CDF854801599491C159121
:101370008142FAD330880D9908440D9070880E99F7
:1013800008440E90B0880F9908440F90F0880C998B
:1013900008440C9001212846FFF7CCFCBDF82C0036
:1013A000401CADF82C00BDF82C00A042DAD30D98FB
:1013B000354A40F3CF1633480A3006830E9941F37D
:1013C000CF1444830F9941F3CF1383830C9941F3D6
:1013D000CF1CA0F804C0ACF5C05C40F2C371ACF502
:1013E0009B7C8C450ED2A6F5C856363E8E4209D25D
:1013F000A4F5C854363C8C4204D2A3F5C853363BFE
:101400008B4203D3D18841F48041D180D1884904F3
:1014100007D41E49028B21F85C2F428B4A80808BB7
:10142000888000212846FFF747FA0021384600F05F
:10143000A7F800212846FFF735FA00214C46484618
:10144000FFF730FA0220C102401C8842FCD3284634
:10145000FFF74EFB2046FFF74BFB384600F09CF8A9
:10146000FFF734FA0A493C20087062B616B0BDE8AE
:10147000F0870000001002400024014000280140D5
:10148000080002402E050020600A0020C00C002049
:101490002007002070B5204B40F6C81441F2B70574
:1014A0005B6C48F6E6065C4305EBA4341B4D7343C6
:1014B0004EF6F61606EBA333C5E90443D460401A92
:1014C000536110609168884202DA4942884200DC28
:1014D000116010684343107E0341906A19189162AD
:1014E000506A814200DD9062916A106A814201DB9C
:1014F000084600E09062A86111684C43117C0C41E1
:1015000008412118B2F91C00884204DBB2F91A0024
:10151000884200DC08B270BD48010020280100208C
:1015200010B54FF40054204600F0ACF8002813D05A
:101530000A49087840F008000870204600F014F8C6
:101540000021074800F01CF80648C17E012903D19C
:101550000021C1760121017710BD00008206002024
:1015600044000240640B0020C10002D5024908601B
:10157000704702494860704704040240000002407E
:101580000029016802D041F0010102E04FF6FE722D
:10159000114001607047000001684FF6FE72114073
:1015A00001600021016041608160C1603149314AC0
:1015B0000839904203D1486840F00F0006E02D4AF8
:1015C0001432904204D1486840F0F00048607047FF
:1015D000284A2832904203D1486840F47060F5E709
:1015E000244A3C32904203D1486840F47040EDE711
:1015F000204A5032904203D1486840F47020E5E719
:101600001C4A6432904203D1486840F47000DDE720
:10161000184A7832904203D1486840F07060D5E7AC
:10162000154A111F904203D1086840F00F0006E0F0
:10163000114A1432904204D1086840F0F00008606A
:1016400070470D4A2832904203D1086840F4706018
:10165000F5E7094A3C32904203D1086840F47040F3
:10166000EDE7054A50329042EAD1086840F4702014
:10167000E5E700000800024008040240406880B22C
:101680007047000001460020CA0001D5034A00E06F
:10169000034A12680A4200D0012070470004024049
:1016A00000000240002A026801D00A4300E08A4399
:1016B0000260704730B5036847F6F07293430C6AD6
:1016C0008A682243D1E904452C4322438C69224392
:1016D000CC6922434C6A22438C6A22431A4302603B
:1016E000CA6842600A6882604968C16030BD0021F2
:1016F000016041608160C160016141618161C161DE
:10170000016241628162704710B5114C8CB00021BA
:101710002046FFF735FF2046FFF73EFF0D480090BB
:101720000D480021CDE901016420CDE903018020AD
:10173000CDE905010791089109910A916946204672
:10174000FFF7B8FF01212046FFF71AFF0CB010BDCC
:101750005800024004380140BC07002010B50121A8
:101760008CB0084602F072FB1E4C00212046FFF7A9
:1017700007FF2046FFF710FF1B4800901B48019011
:1017800000211020CDE902018020CDE9041006914E
:101790000791089109910A9169462046FFF78AFF4F
:1017A000012202212046FFF77DFF01218DF82F1035
:1017B00004208DF82D008DF82E100E208DF82C00B1
:1017C0000BA802F04BF80F208DF82C000BA802F0AC
:1017D00045F801212046FFF7D3FEFFF795FF0CB037
:1017E00010BD0000440002400438014058070020AA
:1017F00030B540F6AA21204AC184838B1488E31AAD
:101800009BB20F2B10D312888283037E002253B128
:101810001A4BB3F90A30062B05DB194B1B78022B48
:1018200003D0002B00D1828430BD164B40F68B25AF
:101830005B6CA3F22D14AC420FD2428B521C92B2BD
:101840004283642AF0D364224283B0F924208A427E
:1018500001DA02EB2111818430BD41F29414A342DC
:10186000FADBB0F92430002B02DDA3EB211100E0FC
:1018700000218184428330BD2C07002064000020B9
:10188000230700204801002010B50446B0F90200EB
:1018900043F6991148438113E06840F26662504371
:1018A00001EBA030E060B4F9001043F69912514307
:1018B0008A13216940F26663594302EBA131216129
:1018C00004F08AFE6061A18840F6AB220844401013
:1018D000A0F515415539E062914205D9A0F5F851BE
:1018E000FF39521C91421DD249F25451884202DD07
:1018F000A0F5204002E0A0F5F850FF38206300EB8F
:10190000400040F34F002085B4F924104A42904231
:1019100001DA104602E0884200DD0846E0832284B6
:1019200061848AE0A0F5FE42FF3A41F255518A42B5
:1019300014D8A2F6AA20206300EB400040F34F0029
:101940002085B4F924205142E183884201DA084617
:1019500002E0904200DD1046404250E0A0F5D44243
:10196000AA3A8A4215D2A2F6AA20206300EB4000D0
:1019700040F34F012185B4F924004242E2832084E0
:10198000914201DA104602E0814200DC08466084A0
:1019900053E0A0F5AA42543A41F256539A4215D266
:1019A000A2F6AB20206300EB400040F34F002085FF
:1019B000B4F924104A42904201DA104602E088420B
:1019C00000DD08464042E083218419E0A0F5804212
:1019D00041F254539A4215D2A2F6AA20206300EB9A
:1019E000400040F34F012185B4F92400E0834242D6
:1019F000914201DA104602E0814200DC0846208470
:101A000062841AE0A0F52852AB3A8A4215D2A2F6B7
:101A1000AA20206300EB400040F34F012185B4F978
:101A20002400E08342422284914201DA104602E01F
:101A3000814200DC08464042A9E7B4F91E00A0EB51
:101A400040208013E080B4F92000A0EB40208013F8
:101A50002081B4F92200A0EB40208013608110BDEA
:101A600001210176704770471548164A4FF48041AE
:101A70000078042821D002F13C03D08A9B88C01A48
:101A800000B22F2801DD001108E0002801DD002050
:101A900007E00D4B984201DA184602E0402800DDCD
:101AA00040209389184400B2884203DC40F266610A
:101AB000884200DA084690817047918170470000A3
:101AC00023070020D0040020C0FEFFFF38B54B489C
:101AD0004B4902880B889A1A92B20F2A71D309884F
:101AE000484C01804FF0FF01E2884FF47A735504AF
:101AF0004FF4967002D51622009103E0950403D5A9
:101B000015220091014670E0D50402D514220091FF
:101B1000F8E7150502D513220091F3E7550502D524
:101B200012220091EEE7950502D511220091E9E716
:101B3000D50502D510220091E4E7150602D50F2243
:101B40000091DFE7550602D50E220091DAE79506EF
:101B500002D50D220091D5E7D50602D50C220091C1
:101B6000D0E7150702D50B220091CBE7550702D528
:101B70000A220091C6E7950702D509220091C1E724
:101B8000D20702D008220091BCE72289550702D56E
:101B900007220091B6E7950702D506220091B1E72A
:101BA000D20702D005220091ACE7A27AD20702D078
:101BB00004220091A6E7A289D40603D5032200914E
:101BC000A0E719E0140702D5022200919AE7540712
:101BD00003D4940701D4D20702D00122009191E7E7
:101BE0000020034602460146009002F037FFBDE8A0
:101BF00038400248FFF756B938BD0000540A0020AB
:101C00002C070020600A0020F0B559485949828805
:101C10000B889A1A92B29C2A64D30988818056490B
:101C20000A880146002A0B7843F0020156D1164675
:101C3000524A1C0715680246127822F0020274D537
:101C40004F4C0746E4887F785FEA845C02D547F012
:101C5000010701E027F001074770A704477802D584
:101C600047F0020701E027F002074770670401D43C
:101C7000E70703D0477847F008074770640603D5A5
:101C8000447844F0040404E01C0603D4447824F0AF
:101C900004044470EC0450D4354C9A07247824F0A2
:101CA000100423D4324D42782F7A2D78012A45F042
:101CB000100514D0022A16D02D4C042AA47804F161
:101CC000010C0CF0FF0C13D0072A25D0032A23D0D7
:101CD000052A21D0062A1FD021F0100142E0B907C1
:101CE00002E00570F0BD39070029FADB0470F0BD91
:101CF000FA0601D41A060AD50170022C04D280F823
:101D000002C0BCF1020FF2D341F080012AE021F0C1
:101D1000100101708670F0BD877A7F06F7D5032C1D
:101D200004D8017080F802C0F0BD0FE05107D8D58B
:101D30001906D6D443F0800114E002704178CB0735
:101D400001D18907F0D522F010010BE0E9040BD492
:101D50009907E9D4818AC82902D2491C8182E3E724
:101D600043F00A010170DFE702708682DCE70000C1
:101D7000040700202C0700202E070020AC020020C2
:101D8000600A0020094944F648000880091D46F60B
:101D900048000880091D41F6CC4008800348001F18
:101DA000018841F02001018070470000182C01409B
:101DB000084946F668000880091D0880091D41F29F
:101DC000555008800348001F018841F02001018020
:101DD00070470000182C014010B5C28800210AB1DC
:101DE000032206E002890AB1022202E0428912B10E
:101DF0000122027000E0017004784FF4804344F641
:101E0000206244B1012C06D0022C07D0032C01D152
:101E10004180818010BD4380828010BD41F233310A
:101E2000418040F6B731F4E730B5B1F86A5000238D
:101E30001A240D22854202DCB1F9680030BD4D88BC
:101E4000854202DBB1F9000030BD01EB82056D88EF
:101E5000854201DD144601E013DA134604EB030268
:101E60004FEA52029A42F0D101EB830231F823107B
:101E700054889288521A001B424301EB622000B240
:101E800030BD31F9220030BD054920B1086940F06C
:101E90008000086170470348486003484860704705
:101EA0000020024023016745AB89EFCD06494FF47E
:101EB0007A70CA68D20705D0401E0004000CF8D121
:101EC000FF20704700207047002002400E4A032088
:101ED000A2F1500182F83E00002048810B4908869B
:101EE000C862C8830884488490620948016DB1F5CE
:101EF000206F01DBA3219162807A002802D0906AD2
:101F000040429062704700006400002038050020C5
:101F1000480100200449002048810881C862886285
:101F2000024988627047000064000020CC0800204D
:101F3000F0B53B4988894A89801A80B20F2866D358
:101F400088894881CA8937480B3A272A26D28A7855
:101F500022BB8268364B42F480728260324A354C32
:101F6000354D12785607314A0AD4344E36881680D9
:101F7000334A12881A80334A12882280324A09E092
:101F8000324E36881680324A12881A80314A1288B8
:101F90002280314A12882A8001228A702F4B304DCC
:101FA00019469A7F0968802A32D302F01F0255F839
:101FB000222011422CD0826822F48012184E8260B6
:101FC000123614461215B778521C62F38617254A4A
:101FD000B77093F816C01778BCF1800F27F002068F
:101FE00008D30CF01F0C55F82CC011EA0C0F01D1CE
:101FF00047F0020616701A7E802A0DD302F01F02E7
:1020000055F82220114207D144F400218160F0BD2F
:10201000826842F48012D1E724F40021F6E7000040
:1020200020070020AC02002048010020C804002046
:10203000CA040020CC040020CE040020B8040020F4
:10204000BA040020BC040020BE040020C00400200C
:10205000C2040020C4040020C6040020E8050020BB
:102060003C930008D004002070B520488189028983
:10207000891A89B20F292FD3818901811C4B1D48F0
:1020800019465D7A06681C4C096846F00402802DEA
:1020900007D305F01F0554F82550294201D126F039
:1020A000040202609A7B802A17D302F01F0254F8C0
:1020B0002220114211D1026822F002020260DA7A73
:1020C000802A0ED302F01F0254F82220114208D1B8
:1020D000016821F00801016070BD026842F002024F
:1020E000ECE7016841F00801F5E700002007002057
:1020F000E8050020AC0200203C930008F0B51D4C20
:102100001B4A4FF0010C94F83B5094F80AE0144637
:1021100092F83C3094F838402B43651CEEB2154DD4
:1021200095F83D700025BEF1FF0F0AD0BEF1000FFB
:1021300006D18B4213D155700C2C01D282F8386035
:10214000F0BD834202D182F801C0F5E78B42F7D19E
:102150005570B80709E000BF82F83850F0BD8342DF
:10216000FCD1F84382F801C080070028F4D0F0BD0C
:102170005804002048010020F0B5CA78002502F07C
:102180000F03D20601D58A7813430A784FF00F0E59
:1021900012F0FF0F4FF001021CD004680F8802FA02
:1021A00005F63740B74211D14FEA850C0EFA0CF70D
:1021B00024EA070703FA0CF43C43CF78282F02D017
:1021C000482F02D002E0466100E006616D1C082D38
:1021D000E4D304600C88FF2C1ED944685FF000062D
:1021E00006F1080702FA07F50F882F40AF420FD11A
:1021F0004FEA860C0EFA0CF7BC4303FA0CF73C438B
:10220000CF78282F00D14561CF78482F00D10561C4
:10221000761C082EE4D34460F0BD0000F0B5144CE9
:10222000002801DAE36900E06368420D120185B21B
:10223000C0F301579540C0F30346032F05D0C202F7
:102240000AD50322B240934307E023F0706263682B
:1022500023F07063636002E0AB4343F0706201B14E
:102260002A43002801DAE261F0BD6260F0BD00009F
:10227000000001400246002092680A4200D001207E
:10228000704741617047016170470AB10161704751
:10229000416170470F4A104B92F838105B5C8342E3
:1022A00001D1012004E00D4B5B5C834203D100208F
:1022B00082F83A0070470A4B5B5C834201D181206F
:1022C000F6E7084B595C814201D18020F0E70320FA
:1022D000EEE7000048010020F49700080698000887
:1022E000FA9700080C9800080A4810B501784FF0DA
:1022F00000024C0708494FF0FF0389684FEA01715B
:1023000005D5002901DA827210BD837210BD002943
:10231000FBDBF8E748010020AC020020F0B5194EC5
:10232000194C0022E31CA6F1060CB75CA518ED7849
:10233000FF5C0D430F43BD421FD01CF80270FF5CD1
:102340000F43BD4219D015460023A618F6780E4358
:10235000C6545B1C1CF80220DBB2062BF5D3C178F7
:1023600081700179C17000214218491C15711CF857
:102370000550C9B20629F7D3F0BD521CD2B2032AC8
:10238000D3D3F0BDCE8E00085804002010B502460D
:102390000021064B06205C186478944200D1084660
:1023A000491CC9B20629F6D310BD0000480100201F
:1023B000214810B590F8671000222048012936D135
:1023C0001F49898899BB1F491E4B4C6C40F6B83198
:1023D000B3F876308C4227DD1B49097821BB90F891
:1023E0002711491CC9B280F82711C8291CD380F8CD
:1023F00027210146D0F82C4191F82811A34203DD92
:10240000052908D2491C01E041B1491E80F8281174
:10241000C9B2052902D3012180F82611191B074CE6
:102420002C3C6162C0F82C31B3F5FA6F03D280F80E
:10243000262180F8282110BDC00C0020AC0200200D
:10244000E205002048010020230700204FF4C0428D
:10245000C260002181620E22028241F26202426168
:10246000082202834FF46042428381834FF0784216
:10247000C0E9082140F6C41101807047B0F900108E
:10248000B0F90220891A41604269037E4A431A4129
:10249000836A13448362426A934200DD8262836AE4
:1024A000026A934200DA8262C268836A4A43017C0C
:1024B0000A410B41D118B0F91C208A4201DA1046BA
:1024C0007047B0F91A008842FADC08B27047000081
:1024D00010B514481449B0F894200B889A1A92B297
:1024E000B2F5437F1DD90988A0F89410B0F8921076
:1024F00020F8601F002242860C480D4CC288828062
:10250000C180C38983812489891AA4B2C48181606E
:10251000E11A0161074A818AC182928A8282511A34
:10252000816110BD480100202C070020880C00208C
:10253000380500206400002009480A49B0F8B2209C
:102540000B889A1A92B241F684639A4206D309889C
:1025500020F8B21F4188818000214180704700002F
:10256000480100202C0700200D480178C90702D03F
:102570000C49098801E04FF6FA71416609490120CA
:102580001039088007482438018841F00101018092
:1025900004481838018821F01801018070470000B4
:1025A00048010020240400400A49D1F8982012B1C3
:1025B000521EC1F8982031F8922F521C21F81A2986
:1025C0004A6A521C4A628A8F521C8A8701F8400C60
:1025D00070470000480100201CB52D4890F83B30A2
:1025E00090F83C20934252D000248DF80440534090
:1025F0008DF800309DF800300122012B08D09DF8A5
:102600000030022B09D09DF80030042B0AD00DE0D9
:102610001F498DF80420443108E01D498DF804203D
:10262000463103E01A498DF8042048319DF8042012
:10263000012A2CD190F83D309DF80040154AA34264
:1026400017D090F83E309DF80040234208D0B0F8F3
:102650004C30A0F84A300B881488E31AA0F84C30AC
:1026600090F838302BB1B0F840301488E31AA0F855
:10267000423012880A80A0F8402010F83E1F9DF8D2
:102680000020114300F801199DF8001001701CBDD5
:10269000580400202C07002070B5344D40212846F6
:1026A000FFF7E8FD840080212846FFF7E3FD44EAB8
:1026B0004004A9152846FFF7DDFD0443E1B22C4C88
:1026C00094F878508D4250D04D4084F87810012D08
:1026D00003D0022D01D0042D47D194F87C00A843EB
:1026E00084F87C0094F87B20AA420FD084F87B50B9
:1026F00094F87A2001238B401A4207D11A4384F8B8
:102700007A2094F87910491C84F8791094F879109B
:10271000042928D330B1012811D002280FD0042871
:102720000DD012E01348C18821F04001C18020780B
:10273000002184F83B1020F06000207005E0217833
:1027400041F02001217084F83B000B4994F83B00D4
:1027500091F82720904204D081F8270007492020D3
:10276000087000F00DF884F8545070BD001001405E
:1027700048010020600A0020C00C00202007002033
:1027800070B50D4D40212846FFF774FD840080216F
:102790002846FFF76FFD44EA4004A9152846FFF7D5
:1027A00069FD04430548072100F8784F01710021B5
:1027B00041708170C17070BD00100140480100205F
:1027C00070B5344890F83A10CA43920761D001F0CE
:1027D000030280F8392090F83D305B061B0E80F82C
:1027E0003D30012A01D0812A02D15B1C80F83D30A6
:1027F0000278D2074DD0DBB203F00102C3F34004EC
:10280000A24246D1B0F856400025641CA0F85640BC
:10281000204CA0F8585090F83E60A47AB24202D002
:1028200080F83E200DE0A607B6EB837F02D080F84B
:102830003F5006E090F83F30642B02D25B1C80F8DA
:102840003F3090F84030642B0CD25B1CDBB280F838
:102850004030022B06D204F00103934202D102223F
:1028600080F84020012901D0002912D190F83820A9
:10287000416E00EB820291610163D0E906121144BE
:10288000D0E908231A441144826A1144C26A1144EF
:10289000416370BD48010020FEE700002DE9F04FC4
:1028A00000BF00209E4E9F4AA6F51271A6F5BE7984
:1028B000A6F1440B06F1440E804601F5E074A1F147
:1028C000780301F5457A1D5C15F0C00706D0402F4E
:1028D00051D0C02F77D0802F76D004E115F01F059E
:1028E00004D0154440F080072F7201E082F8088080
:1028F000012826D0022824D0032822D0042820D062
:1029000008281ED010281CD0874D55F820C0DCF8B0
:10291000005054F820703D40CCF80050824D55F8DE
:1029200020C0DCF8005056F820703D43CCF8005031
:102930001D5CAD0659F820502F6813D53AF810C029
:102940003EE051F820502F6854F820C007EA0C07E9
:102950002F6051F820502F6856F820C047EA0C0726
:102960002F60E5E7DFF8B8C10CF1F00C5CF820C08F
:1029700007EA0C077EE015F01F0504D0154440F06F
:1029800080072F7201E082F8088001281DD00228FC
:102990001BD0032819D0042817D0082815D01028D8
:1029A00013D0614D55F820502F6854F820C007EA25
:1029B0000C072F605C4D55F820502F685BF820C045
:1029C00047EA0C0756E00BE056E051F820502F681C
:1029D00054F820C007EA0C072F6051F82050ECE7AC
:1029E00015F01F0505D0154440F0800785F82170CB
:1029F00001E082F82180012825D0022823D0032875
:102A000021D004281FD008281DD010281BD0464DE7
:102A100055F820C0DCF8005054F820703D40CCF848
:102A20000050414D55F820C0DCF800505EF8207091
:102A30003D43CCF800501D5CAD0615D53A4D3AF833
:102A40001070CC3514E051F820502F6854F820C095
:102A500007EA0C072F6051F820502F685EF820C05D
:102A600047EA0C072F60E6E72D4D3AF81070E03D7D
:102A700055F820502F6036E015F01F0505D015449D
:102A800040F0800785F8217001E082F8218001285C
:102A900030D002282ED003282CD004282AD0082891
:102AA00028D0102826D0204D55F820C0DCF8005042
:102AB00054F820703D40CCF800501B4D55F820C014
:102AC000DCF80050164F883757F820703D43CCF89B
:102AD00000501D5CAD06B1D4114F3AF81050E03FE4
:102AE00057F820703D60401CC0B21128FFF4EBAED7
:102AF000BDE8F08F51F820502F6854F820C007EA45
:102B00000C072F6051F820502F68DFF814C00CF12B
:102B1000880C5CF820C047EA0C072F60D9E700005A
:102B2000C8950008E8050020C49300084FF4077119
:102B3000C1824FF45861018340F61451818370477C
:102B4000F0B5C48AB0F900608681B0F90250C58141
:102B5000B0F904300227002101220382AB4204DBDA
:102B6000B54202DDC78042810CE0B34204DBAE42D5
:102B700002DDC78041811CE09D4205DBB34203DDDD
:102B8000C2804781018115E0B54204DB9E4202DD2F
:102B9000C280418105E0AE4205DB9D4203DDC1807C
:102BA0004281078106E09E4204DBAB4202DDC18028
:102BB00047810281C388458900EB430700EB450547
:102BC000BB89AE899B1B0FFA83FEA0F812E0068931
:102BD000AB8900EB460CBCF80CC0A3EB0C03838262
:102BE000B0F91830B7F90CC0A3EB0C0CB4EB4C0FD8
:102BF00004DA80F82010A3F1A10113E0A64503DD5B
:102C000080F82010B9890BE026B1012E04D0022EE5
:102C100010D004E0062100E0052180F82010A989E9
:102C2000091B6D31418309B2B1F5586F04DB5B1E9E
:102C3000438304E00421F0E7002900DC4283418B58
:102C40008183F0BD0B49002288760A62CA614A621C
:102C5000094A32F9103002EB40028B62B2F90220CD
:102C6000CA62064A32F810000882A1F86000A1F892
:102C700062007047000200201E98000812980008A9
:102C80002DE9F05FFA48FB4982880B889A1A92B2C4
:102C90000F2A44D309888180F749814601240A8894
:102CA000F648F74E00257AB3521E0A80C573F54ADE
:102CB00085620168B2F902204F0742F6AA2318D4B0
:102CC000F78847F40057F780EE4E3678B60709D5F7
:102CD000866826F080068660A0F87C5080F87E50DA
:102CE00080F87F50CE0404D480F8F040C0F8EC5057
:102CF00003E080F8F0504E0707D49A4205DB80F8D5
:102D0000F440A0F8F25004E010E080F8F4504E07D0
:102D100003D49A4201DBC90703D080F81151BDE802
:102D2000F09F80F81141A0F81251F8E78046B0F802
:102D3000181143F69820814202D2491CA8F81811B4
:102D400001F0A2FED04FDFF828B397F85000ABF1A6
:102D50001C0B10B1FEF7B0F905E09BF8001021F054
:102D600001018BF80010FFF723FB00F0D1F9C748F1
:102D700041F26801426C4FF400608A4201DBC449B1
:102D800004E0B2F57A6F02DAC149091D086097F8CC
:102D90005100DFF8E8A2BF4BBF4FC007AAF12C0AD1
:102DA0003AD0987B802833D398F8001089072FD425
:102DB00098F80F008AF80500B248514690F800C014
:102DC0002CF0020C80F800C0ABF80250CBF8145085
:102DD0009BF800C02CF0010C8BF800C0B0794006C5
:102DE00011D44889B0F5FA7F03D2401CAAF80A0032
:102DF00012E040F63C70824201DD00200FE1082025
:102E00008AF803400BE1CD700020AAF80A5006E1D1
:102E10008AF80350AAF80A50D8F80800010501D52D
:102E20000820FCE0984991F83FE05FEACE7149D074
:102E3000984B98F80F208AF805205B7A4146802B42
:102E40004CD30B785B0735D4F3889B0405D500BFC2
:102E500020F02000C8F8080034E0ABF80250CBF8AE
:102E600014509BF800C08B4B2CF0010C8BF800C069
:102E700040F020008860D87D80280AD300F07F0CC5
:102E80001B684FF0004020FA0CF0034201D10C7196
:102E900000E00D710879C00702D15FEA8E7005D598
:102EA0000320032A01D08AF80840B8E00020C8F8BF
:102EB0002850B4E020F02000C8F80800F08820F482
:102EC0000050F08098F82601444601280BD06E4847
:102ED00090F8630048B1FDF7AFFF0FE00A6842F0D9
:102EE00004020A60B4E7092099E0A068C10502D590
:102EF00020F0080001E040F00800A06094F84600CF
:102F00004FF4804198B1012817D00228387823D097
:102F1000C0F38102881E012A28D0022A26D0A4F8F4
:102F200014115E4890F85E00042822D016E043F2A7
:102F30001E5000BFA4F8140110E0387842F6CC42CD
:102F4000C0F38100012804D0022802D043F2EB1024
:102F5000F0E7A4F8142101E0A4F81411A4F8441037
:102F6000494890F87000012808D017E0A4F814012F
:102F7000D7E743F69910A4F84400F1E7387842F215
:102F80006662C0F3810001280FD0022810D041F6FC
:102F9000E12000BFA4F81401A4F844209BF800200D
:102FA000D20708D0BBF8022007E0A4F81421F3E709
:102FB0004FF40050EEE733488288A9F8122010B28F
:102FC000B4F944205043C0F38F325046AAF812207F
:102FD0008A4200D9418232490978C90605D5428A18
:102FE00041F233318A4200D241822189C1F3C002C9
:102FF000C1F300218A4205D1428A41F699118A42E1
:1030000000D94182B17AC90700D04582BAF81200CE
:10301000A06200287FF7F1AE22480570022099F8DF
:103020001A1099B902283FD080B1184A11788C063D
:1030300008D5B479640605D5194C2478E40964F3FD
:1030400086111170F18821F40261F1800F49496CF9
:103050004E2907DBB179090604D50A490A7822F01E
:1030600002020A7089F81A0088F80F0057E600007B
:103070006C0900202C0700202E070020AC02002045
:10308000600A0020E2050020C00C0020480100205A
:10309000100C0140E8050020D0040020640000204E
:1030A0000407002040070020398F0029BDD143F6D6
:1030B00098213987B9E770B500230C8863F30F02B4
:1030C000012505FA03F6344206D0C3F10F0605FACE
:1030D00006F1114361F30F025B1C102BF1DB028040
:1030E00070BD70B500230C7863F30702012505FA63
:1030F00003F6344206D0C3F1070605FA06F1114380
:1031000061F307025B1C082BF1DB027070BD00004D
:10311000F0B51F4890F866301E48012B816821F4F5
:10312000006232D11C4BDE8874062ED41B4D0F0575
:103130004FF00004B5F902501ED4194A526C642AAB
:1031400011DC40F6386295420DDAB2040BD40278F5
:1031500052070ED4B0F8D42040F6B835AA4203D2B4
:10316000521CA0F8D420F0BD41F4006181605C8164
:10317000F0BDA0F8D440F0BD41F2CD018D42FADDA2
:10318000997AC907F7D18260F3E78260F0BD000049
:10319000C00C0020AC020020600A0020E2050020E4
:1031A000480100200C490D484B88426C03B98264E9
:1031B0005B1C9BB24B80FA2B0CD3836CD21AC2647B
:1031C0000020488040F6B830824203DB04490120E9
:1031D00081F80D01704700006C09002048010020B3
:1031E000AC020020F0B5364D364F044695F83B0052
:1031F00097F83B1023780843EE1C6278834205D190
:10320000E0781146FEF77AFF207908E094F802C0D2
:1032100084450CD1E1781046FEF770FFE07905F89F
:103220002F0F2878805D6870287BE877F0BD824298
:103230001DD161461846FEF761FF95F84E1095F8CE
:103240003B00814207D1B97A09B1A17900E06179E7
:1032500085F82F101EE06978012901D0A17922E0BC
:10326000617927E0297841F00401297012E0E178C2
:103270008142DBD119466046FEF740FF95F84E10BB
:1032800095F83B0081420AD1B97A09B1617ADFE74A
:10329000217ADDE715F82F1F895D6970C5E7697828
:1032A000012906D0617A85F82F10B97A0029F1D169
:1032B000D8E7217A85F82F10B97A0029EAD0D1E72A
:1032C00058040020480100200B48017821F0020139
:1032D00000F8381B002100F8181941778177332155
:1032E0008185418508214184012100F81F1C034884
:1032F00080F8391070470000580400204801002071
:103300000D4900B50B4851F8012F40F8032F89886B
:103310008180084801210930FFF700F805480221A3
:103320001330FEF7FBFF034804211D305DF804EB6A
:10333000FEF7F4BF5804002048010020094944F674
:1033400048000880091D46F648000880091D41F222
:10335000111008800348001F018841F020010180FE
:1033600070470000182C01402DE9F047664C674B70
:103370000025A0780126654A103305287ED2DFE8B3
:1033800000F00313113E1100108820F0010010809E
:103390001D805F480580001F0580001F0580FFF726
:1033A000CDFFA670BDE8F087594941F244401C3971
:1033B0000880574945F6580024390880091D47F20E
:1033C0005800088052492020283908800020401CDD
:1033D000C0B27328FBD3FFF7B1FF4C4984F85C50AF
:1033E0002C3147F6906008804848143006801D80D4
:1033F000108840F0010010800220A070D2E7002168
:103400005FF0010004EB410204EB4003B2F85020EE
:10341000B3F850309A4200D20146401CC0B2062890
:10342000F0D33C48405C84F83900FFF74DFF1D2085
:1034300000F0F3F900F076F8374E38484FF4807911
:1034400096F83B10012904D002291BD0042930D062
:1034500047E040218046FEF70DFF8700802140466F
:10346000FEF708FF47EA400749464046FEF702FFDD
:10347000074347F0010084F83B0000E03DE02248AC
:1034800009302CE040218046FEF7F4FE87008021C1
:103490004046FEF7EFFE47EA400749464046FEF742
:1034A000E9FE074347F0020084F83B00164813305A
:1034B00015E040218046FEF7DDFE87008021404672
:1034C000FEF7D8FE47EA400749464046FEF7D2FEDF
:1034D000074347F0040084F83B000B481D3002F01E
:1034E00033FF94F82F0086F838001D2000F0ABF968
:1034F0000420A0700A48057054E7108820F00100ED
:1035000010801D80A5704DE7580400200008004081
:103510003C2C0140D48E00084801002000100140DE
:10352000230700202DE9F041344C14F82F0F344DBF
:10353000E07240212846FEF79DFE86008021284645
:10354000FEF798FE46EA4006AF1539462846FEF7D4
:1035500091FE0643207BF1B22F3C814215D084F8C6
:103560003C0040212846FEF785FE86008021284643
:10357000FEF780FE46EA400639462846FEF77AFE08
:10358000064384F83B60FFF727F81E4D95F83B0093
:10359000012827D0022828D0042829D0174894F8D9
:1035A0003B102730085C04F8300F14F80109FEF7CF
:1035B000EDFE04F82F09A87A00B10120607001F037
:1035C000FBFA94F84E0094F83B10884206D094F829
:1035D0003800062802D2401C84F8380084F84E10C7
:1035E000BDE8F0810548093004E00448133001E0EB
:1035F00002481D30BDE8F041FFF7F4BD580400203B
:1036000000100140480100202DE9F041524991F895
:103610007200AA287ED191F8730055287AD14F4CB8
:1036200000200A5C2254401CC0B27428F9D34C4ECE
:103630002069C6F80100A08AA6F80500D4F8160093
:10364000F060D4F81A003061D4F81E0012347061B2
:1036500002F020FE4349608A888102F035FE207D19
:10366000123CC007307802D040F0040001E020F0A6
:1036700004003D4930704FF480403C4D886114F89F
:10368000280F85F82000608B6880A08BA880E08BD5
:10369000E880208C2881608C354F688194F8240064
:1036A00087F8D20014F8011C304686F83B1000263B
:1036B000C0F89C60FFF724FE2E48A18E0183E18EA6
:1036C0004183218F818394F84210283C012908D03E
:1036D000022901D0032909D0297821F00C010831F1
:1036E00007E0297821F00C01091D02E0297841F05A
:1036F0000C01297094F86E20012162B1012A01D0D9
:10370000022A0BD087F8461094F864301A4A4BB15D
:10371000518108E014E087F84660F5E7022287F857
:103720004620F1E7568194F8701001290AD094F8E8
:103730006D1051B101290BD04FF48051A0F87610D3
:10374000BDE8F08144F21C71F8E74FF40051F5E751
:1037500041F25551F2E7000000FC0008C00C0020C7
:103760004801002064000020580C0020D0040020F4
:10377000AC02002038050020600A00207CB5012141
:10378000082000F087FB4FF48070ADF8040010248F
:103790008DF8074001208DF8060001A91548FEF7B5
:1037A000EBFC0121092000F075FB01211248FEF716
:1037B00035FD0820ADF8000004208DF803000F4E01
:1037C00003258DF8025069463046FEF7D5FC0821E6
:1037D0003046FEF756FDADF800408DF803408DF8F9
:1037E000025069463046FEF7C7FC10213046FEF70E
:1037F00048FD7CBD0014014000023000000C014077
:10380000FEE7704700F01F0201219140400980004F
:1038100000F1E020C0F88011704700F01F02012184
:1038200091404009800000F1E020C0F8801170470D
:1038300000F01F02012191404009800000F1E020CA
:10384000C0F80011704700F01F02012191404009AB
:10385000800000F1E020C0F80011704770B50F2320
:10386000C47801780122F4B1144C2468457804F43A
:10387000E064C4F5E064240AC4F10406E3408478FB
:10388000B5401C402C4301F1E021230181F80034B4
:10389000007800F01F018A404009800000F1E0201C
:1038A000C0F8002170BD01F01F008240480980006F
:1038B00000F1E020C0F8802170BD00000CED00E0B8
:1038C0000249084302490860704700000000FA05F9
:1038D0000CED00E02DE9F05F00261D20FFF792FFC0
:1038E0006C4CDFF8B4B1A4F1B800A77E90F83810A2
:1038F000DFF8A8E1DFF8A8A100258F427ED0E776A7
:10390000A176626A036B5A434FEA12499BF808207A
:10391000120702D51EF8012000E00A4694F812C0F2
:10392000BCF1010F09D004EB4206B6F902C0C4F89D
:1039300028C0B6F90460E6620CE043F6FF7CC4E9F7
:103940000A5C90F83DC05FEACC7C01D012B102E085
:10395000052A00D1012600EB47074FF0804CBF89B4
:103960003F04B7FBF3F3E361476BBCFBF7F7276258
:1039700094F813C0BCF1000F06D0BCF1010F05D0C4
:103980003B4403EBD3735B10636201E03B46676229
:10399000DFF810C14FF6FF7707EA8307ACF808702D
:1039A0009AF8007090F80A8090F83DC0082F08F04F
:1039B00003070CF0030C05D067450BD1B8F1000FDD
:1039C00005D008E0674505D0B8F1000F03D05B4291
:1039D000636200E06562C6B1636A002B03D006DD56
:1039E000228D05E00AE0304B33F8122000E0A28D72
:1039F000A4F86020227822F0200222709AF8002099
:103A0000042A07D0082A05D012E0B4F8603003EB8E
:103A10000902EDE780F8405065629BF80800000756
:103A200001D51EF80110204830F81100A4F86000FC
:103A30001E49606A09883E314843B4F8601001EBC2
:103A4000204006B21D20FFF7F3FE606A002807D071
:103A500021784FEA81600ADD002804DAA08D09E0B0
:103A6000B4F8600006E0E06AB04208DB0CE0002831
:103A700002DA208D208208E0A06AB04204DD2082B4
:103A800041F02000207000E02682257565752586AE
:103A9000BDE8F09F00020020AC0200200098000862
:103AA00023070020380A0020129800082404004050
:103AB00043184FF48042934210DD904202DD1046DD
:103AC00000210BE0914202DD0020114606E0800358
:103AD000B0FBF3F000B2C0F5804109B241EA00400A
:103AE0007047F0B541F286230022C3600E24826243
:103AF00004824CF2E82508264561068343F6FF77E9
:103B00004283878340F2492E4FEA873CC0F808E0A1
:103B1000C0E9082CCB608A620C824D610E834A8317
:103B20008F83B4208860C1E9082CF0BD0021816238
:103B30000949C1600E2101824FF6BF514161082140
:103B400001834FF44041418343F6FF7181830907AC
:103B50000162024941627047638A010000C0FF0FA1
:103B6000064941F6A260088005480168054A01F44B
:103B7000E06111430160BFF34F8FFEE7442C014029
:103B80000CED00E00400FA0538B501210D2000F02D
:103B900081F94FF4E060ADF8000018248DF803407F
:103BA00003258DF8025069460D48FEF7E5FA4FF4FB
:103BB0006040ADF800008DF803400A4C8DF80250CB
:103BC00069462046FEF7D8FAA014ADF80000482058
:103BD0008DF8030069462046FEF7CEFA38BD000096
:103BE00000080140000C01402DE9F0410121CE0206
:103BF0008CB0304600F04EF9DFF86C81404601F0A1
:103C000051FC08A801F07AFE4FF45860ADF824008A
:103C10000024ADF820402020ADF822000125ADF8A9
:103C200026408DF8285008A9404601F019FE0021D1
:103C3000404601F06CFE4FF6FF71404601F071FE08
:103C400001220021404601F0FDFD0121404601F026
:103C5000E5FB04A801F0FDFBADF81060A802ADF88B
:103C60001200ADF81440A220ADF816002803ADF8FC
:103C70001800ADF81A40ADF81C4004A9404601F008
:103C8000D7FB6027ADF80070ADF80440ADF80840F0
:103C9000ADF80C40ADF80240ADF80640ADF80A4072
:103CA000ADF80E406946404601F0BCFC694640460E
:103CB00001F0FEFC6946404601F044FDADF80450B9
:103CC00040F61450ADF80070ADF80600ADF80840AD
:103CD000ADF80C40ADF80250ADF80A40ADF80E401A
:103CE0006946404601F072FD0121404601F0BAFBF1
:103CF0000821404601F0D6FC3146404601F018FD4F
:103D00000821404601F05CFD3146404601F090FD3F
:103D10007021404601F099FD18208DF82C008DF897
:103D20002D408DF82E408DF82F500BA8FFF796FDF3
:103D30000D480C30018841F0800101800A481430A0
:103D4000018841F001010180001F048001214046EB
:103D500001F092FB8DF828500121404601F096FBBE
:103D60000CB0BDE8F0810000002C0140704740F22B
:103D700013414160082181608621C1604FF4804178
:103D800001614942416100210162C16270470162E3
:103D90007047000010B501884288891A09B2018372
:103DA000B1F5005F02DBA1F5804104E011F5005F91
:103DB00002DC01F580410183B0F9182041685143CC
:103DC000C1618368846A5343C2681B12624303EB78
:103DD0002222036A1A44114402628A134262416930
:103DE0008A4203DB01698A4200DC11468A1AC0E973
:103DF0000A21028E4FF40373594302EBA13202866B
:103E00000B4A1278082A04D10A4A936F03EBA131B6
:103E10009167B0F93010B1F5804F02DDA1F5804116
:103E200003E0002902DA01F58041018610BD00009F
:103E300023070020740A0020034A516821F44041FE
:103E4000014351607047000000100240044A0029FD
:103E5000516901D0014300E0814351617047000086
:103E600000100240044A0029D16901D0014300E05A
:103E70008143D1617047000000100240044A0029CC
:103E8000116901D0014300E08143116170470000D6
:103E900000100240044A0029916901D0014300E06A
:103EA000814391617047000000100240044A0029DC
:103EB000D16801D0014300E08143D1607047000028
:103EC0000010024030B524494A6812F00C03234A1E
:103ED00003D0042B01D0082B26D002604A680F23A0
:103EE0001F4C03EA1212A35C0268DA4042604B687E
:103EF000072505EA1323E35C22FA03F383604B688A
:103F000005EAD323E35CDA40C2604B68032403F480
:103F1000404104EA933303EB9161114B1B1F595C41
:103F2000B2FBF1F1016130BD4A680E4B1A404B689B
:103F3000140103F4803303D5C2F38342113202E04B
:103F4000022404EB924213B14B689B0301D5064B4C
:103F500000E0024B5A43C0E70010024000127A0012
:103F60000400002000003C0800093D002DE9F0415C
:103F7000274CA61540212046FEF77CF985008021BC
:103F80002046FEF777F945EA400531462046FEF720
:103F900071F90543EDB240212046FEF76BF9870029
:103FA00080212046FEF766F947EA40073146204661
:103FB000FEF760F90743F8B2A842DBD14021204662
:103FC000FEF758F9870080212046FEF753F947EAAB
:103FD000400731462046FEF74DF90743F8B2A842A4
:103FE000C8D140212046FEF745F9870080212046B0
:103FF000FEF740F947EA400731462046FEF73AF916
:104000000743F8B2A842B5D12846BDE8F0810000C8
:104010000010014010B50268416802FB02F301FB89
:1040200001330D4CA34211D91B0E0E3B0B4C9BB21E
:1040300012B234F8133009B25A43594342F38F3263
:1040400041F38F31C0E90221012102E0C0E90221E0
:104050000021017410BD0000E10BBF0E248C00088C
:104060002DE9F05FFE48FF4902880B889A1A92B248
:104070000F2A7DD30988FC4E018043F23332B6F912
:104080001810FA48FA4F0025DFF8E893FA4C9142ED
:1040900013DBD9F8442040F6B8318A420DDC94F89D
:1040A0000D1151B1C18841F08001C180F3490A78F6
:1040B00022F002020A70E5733D7081894A0703D439
:1040C0008A0701D4CA0703D0C28842F4007202E012
:1040D000C28822F40072C2808246080702D4504689
:1040E000C90604D5BAF8061041F0010102E0C18802
:1040F00021F00101AAF80610DC48FDF76DFEE0484A
:10410000B0F93A10B1F5804F02DA491C418703E05B
:10411000DB494FF480404887D9F8501041F6CC4035
:10412000814203DDA06820F01000A060D54802881D
:1041300022B1521E0280E5733D7029E0BAF80600F4
:1041400043041DD4BAF80C20D30619D4120717D48F
:10415000020615D4820613D4020511D4420603D5F3
:10416000C94A127812060BD5420709D4C20500E0ED
:104170000FE105D4020703D4820401D4C00607D599
:10418000C248E573C24A3D70C583158080F82A5045
:10419000E08FDFF800C3A34650B1401EABF83E00ED
:1041A000B648037823F0020303708BF80F500BE03E
:1041B000B248027842F0020202703878012804D135
:1041C0009CF80000062800D13D703878DFF8C8E27E
:1041D0004FF001080A286ED2DFE800F0FEDB05DBB5
:1041E000FDFCDB6DFBFA02F06BF99BF80D015C4600
:1041F00008B9FEF7D7FFDFF880A240F62822AAF11F
:104200002C0ACB46BAF81610491C89B2AAF8161027
:10421000D9F84400904202DAAAF8165015E0984AFC
:1042200040F6CC43D2689A420FDB944A43F6991386
:10423000B2F904209A4208DBB1F5FA7F05D3317850
:1042400019B9AAF8165086F80080944A118869B105
:104250009AF804305B1CDBB28AF80430022B05D3D9
:104260008F4B8AF804501988491C1980E17B092971
:1042700012D002297CD0A4F83051B4F84010A946DD
:10428000D1B141F288354946AAF81690A84220DA01
:104290003078012819D01CE071484430FEF7D6F878
:1042A000FDF714FEDBF84410CAF8281041F27C51E7
:1042B000CAF818105FE2A9E1B08A2086F06A70633C
:1042C000B06A3063A4F8408035E0754831700180F1
:1042D0001180744890F8682040F63A20012A0DD0E9
:1042E000C4F8D81084F8EA10CAF82010B4F93010D5
:1042F00001F21D52824218D8102317E094F82821A9
:1043000002B96949C4F8D81084F8EA80B4F93010C9
:1043100001F21D528242B4F8D80000B202D8102334
:104320001A4605E02023022202E02023102200206A
:1043300000F0A0FB20865B484FF4927390F8681061
:104340005A48012915D0DBF8441040F2DC52914262
:1043500003DAB6F90A209A4215DBB4F8402040F699
:10436000C413521C92B2A4F840209A420BD212E01D
:104370001AE0DBF8442040F2DC518A4209DAB6F94F
:104380000A10994205DA87F8009084F8EA90A0F8BC
:104390001A90BDE8F09F3A4AD268002AF9DC42F64A
:1043A000E0629142EFDAF4E7B4F8301140F6B83247
:1043B000914207D22A4B1C3B1B78DB0702D1491CD8
:1043C000A4F830118BB240F2DC518B4208D804E0E3
:1043D000B6E094E0DBE0D6E0DEE042F6CC4103E07C
:1043E000A4F8302143F26661F167CAF828008AF820
:1043F00007802F4FA4F8405084F8EA50797F564642
:10440000C9B1F87F50B3208DB4F9301000B20A233F
:10441000052200F02FFB2086FD777D77B4F9160189
:10442000B4F91411884257DA1E4991F84D10B1B110
:1044300000F1020052E000B21E4901F0F1FCA4F8C4
:10444000E400A16A814200DA0846164900B2B0824F
:1044500091F84D100029B4F930102DE036E039E024
:104460006C0900202C07002064000020600A002056
:104470002307002048010020AC020020E2050020B4
:10448000380500203007002004070020FC08002029
:104490001E000020240700206802002020000020C9
:1044A00022000020C00C00209AF9FFFFE009002044
:1044B000880C0020168E000802D03623052202E068
:1044C00040F24713362200F0D5FA01E040F2666070
:1044D0002086A3E7083001E003DD801EA4F8160162
:1044E00001E0A4F81611B4F930004FF4804188427D
:1044F00001DD21864DE70028FCDA258649E7D3490E
:10450000DBF8DC2058468A4202D2521CC0F8DC207C
:10451000C27B082A03D1D0F8DC208A420CD33D703C
:104520008168CA0502D521F0080101E041F00801C7
:104530008160CBF8DC502CE7BDE8F05F02F0F2BC04
:104540009BF80F005E46092803D035868BF80F5084
:1045500050E1BF4CE069401CE061022809DD208D7C
:10456000012301B2208B052200B200F083FAE5613D
:10457000A062B848218D0180B9F844104180FDF750
:104580007DFF308605E7BDE8F05F04F00DBA9EF8C8
:10459000000009287DD0FCE68BF80D519BF82821FE
:1045A00062B141F31100CBF8D850AB498203F062FD
:1045B00080108A628103B062A8488162A448C582E3
:1045C000D9F8441041F28830814207DA3078012866
:1045D00004D1A34835700580A2480580A249A34BA9
:1045E0000888401C82B2A2480A80C82A02D30478F4
:1045F000012C17D0B2F57A7F02D30478022C11D0A7
:10460000B2F5FA6F02D30278032A0BD09BF80F00A1
:10461000801E082877D2DFE800F010B0F1EF0476B2
:1046200077A2B6E605700D80BAF8061021F4006195
:10463000AAF8061083F80080E8E7FDF755FE99F820
:1046400000004C46400612D58A48807804280ED0D7
:10465000616C204682290ADA817A94F83D0001F0E3
:10466000030100F00300814201D001F0D9FD387848
:10467000062887D084F83F50206D774940F3110019
:104680008203F06280108A628103B06273488162A3
:1046900000E0AFE0FDF71AFC6D485E4680F8078049
:1046A000BBF81401ABF81601606CABF88250B0F5A2
:1046B000437F12DD4FF48040A6F88000B06840F4DC
:1046C0008060B06094F838100529AAD140F010003D
:1046D000CBF808008CE038705BE64FF48041A6F818
:1046E0008010B16821F48061B16040F28A21884273
:1046F00004DA2078400601D402F000FBB06840F0F4
:104700001000B06074E098E0D9F84400B0F5437F41
:1047100007DA9CF80010062903D000BF8CF800507F
:1047200083E05548017821F040010170FDF7CEFB90
:1047300043F6FE70ABF816010BF1DC04FDF7D4FD77
:104740004E4810F8341F21F00101017043492560E3
:104750008D6241498D6208213970456419E63D48F2
:10476000FDF774FEFDF7B2FB3948D9F844108162B9
:1047700041F27C5181610920ADE79AF80600C0063C
:10478000AAD4D9F844004C46B0F57A7F32DDFDF763
:10479000ABFD2078400611D53648807804280DD02E
:1047A000606C82280ADAA07A94F83D1000F00300C9
:1047B00001F00301884201D001F032FD84F83F503E
:1047C000B4F85000ABF8300001B24FF480405D46C1
:1047D000814200DD2886FDF779FBA86840F48060FF
:1047E000A86094F838100529B8D140F01000A860EE
:1047F000022070E73D70CCE513E0FFE7D9F84400F4
:10480000B0F5437F03DA9CF80010062986D1BAF888
:10481000061021F02001AAF80610FDF765FD04201E
:1048200059E79CF80000062802D087F80080B0E520
:1048300009208EF8000005204DE70E4885708CF8A1
:10484000005086F85E50ABF83050A2E5C0D40100AD
:1048500080020020B0090020CC0800209C08002025
:10486000220000202000002016000020140000205C
:10487000150000205804002032070020740A002090
:1048800030B585B001210420FFF704FB4FF4004050
:10489000ADF8100048208DF8130004A91848FDF762
:1048A0006BFC01210846FFF7DDFA40F68C20ADF8DD
:1048B000040003240020ADF80040ADF80200ADF87C
:1048C00006004FF080456946284600F0C9FF1C20CD
:1048D0008DF80C008DF80D408DF80E4001208DF8FC
:1048E0000F0003A8FEF7BAFF01221146284600F088
:1048F00091FE0121284600F0BFFD05B030BD00004B
:1049000000080140704700002DE9F041304CE0788C
:1049100000285AD12078002857D0401E10F0FF0000
:10492000207052D14FF49670208272B6294F45F212
:10493000AA50A7F872000020FDF7A6FA264D132012
:104940002860FDF7B3FAA8BB3420E8600220286194
:10495000224E6E61286940F040002861FDF7A6FAFA
:1049600040BB00211E4A08465FEA255312F800C0EA
:10497000BCF1FF0F00D00121401C80B29842F5D35A
:10498000C1B9C4E9067639260127A06910F8011BD0
:1049900010F8012BA061E06901EB022102886A6135
:1049A0002F6120F8021BE061FDF780FA10B9761E36
:1049B000B6B2EAD20120FDF767FA62B601F084FCD4
:1049C0000848816821F480418160BDE8F0810000E1
:1049D00020070020C00C00200020024000FC00083E
:1049E00000FC0008AC0200201948016841F01001E9
:1049F0000160016821F003010160016841F00201DA
:104A0000016014484168416041684160416841F477
:104A100080614160416821F47C11416041680E4A27
:104A200011434160016841F08071016001688901B2
:104A3000FCD5416821F003014160416841F0020169
:104A400041604168C1F381010229FAD17047000039
:104A500000200240001002400000280830B5044C3D
:104A6000039D6080A180E2802381658130BD0000CC
:104A7000540A00200A44824201DA10B27047C91A6F
:104A80008142FBDD08B270472DE9F0434348DFF86F
:104A90001081DFF81091C17F457A04680126002358
:104AA000414A424880292BD301F01F0158F82110B8
:104AB0000C420146096802D041F4805101E021F422
:104AC00080510160CF0417D48F0415D5977AFF0762
:104AD00007D0538199F800C02CF0020C89F800C06F
:104AE0000AE090F84670BFB14FF0020C012F18D0C9
:104AF00080F8463080F81AC10F0B67F34D31016022
:104B0000802D2AD305F01F0158F821100C420168AE
:104B10000CD041F004010BE080F8466080F81A31B7
:104B2000EAE780F846C080F81A61E5E721F0040161
:104B300001604C070DD44C050BD5947AE40708D0DE
:104B4000538199F8005025F0020589F80050C0F80B
:104B500098308C0864F38A210160917AC90717D1D3
:104B6000134991F86410012912D11249496C322974
:104B70000CDC0178490709D50189090506D4D0F86C
:104B8000981047F23054A14204D95681C0F89830A9
:104B9000BDE8F083491CC0F89810F9E7E80500204B
:104BA0003C930008E2050020600A0020AC020020CF
:104BB000C00C00204801002010B5FCF7D3F80F48C6
:104BC000018821F0020101800C49183109880C4A42
:104BD000928E1144094A3432118008490C390A88EE
:104BE00042F001020A80011D0A884FF6ED531A4077
:104BF0000A80018841F01201018010BD0C040040C0
:104C00005804002006484188491C89B24180B1F50A
:104C10007A7F04D38188491C8180002141807047BC
:104C2000440700200F4810B5016841F00101016000
:104C300041680D4A1140416001680C4A1140016011
:104C4000016821F480210160416821F4FE01416086
:104C50004FF41F018160FFF7C7FE05494FF0006068
:104C6000086010BD001002400000FFF8FFFFF6FED4
:104C700008ED00E02DE9F0413149324D0888401C33
:104C8000088028884FF00004000629D5FCF7EAF9CF
:104C90002D4A2E4807231778C8262D49012F22D0E8
:104CA0002C4FB7F806C0BCF1000F3ED0B0F80CC0D6
:104CB0004CF0080CA0F80CC0B0F806C02CF4006C46
:104CC000A0F806C0886820F004008860FC8013709B
:104CD000CE8700204FF49661401C80B28842FBD3FF
:104CE0002C80BDE8F0811C4F97F800C0BCF1010F8B
:104CF0000FD0BCF1020F11D0B0F806C04CF4006C1C
:104D0000A0F806C0886840F004008860052038706C
:104D1000DDE7B0F80CC04CF0080C03E0B0F80CC0B4
:104D20004CF0100CA0F80CC0F0E70C4F3C70C7889A
:104D300047F40067C780886840F004008860C6E7D1
:104D400044070020102C014023070020600A0020A7
:104D5000AC0200206C09002024070020410700203D
:104D6000704700002DE9F0434FF08040018A21F0A8
:104D700001010182AB48007800287CD1AA4FF87B62
:104D8000002878D1A948406C322874DCA848806893
:104D9000DFF8A0924104A84DB9F804004FF00004D8
:104DA00003D4401CA9F8040026E1002874D0297817
:104DB000012611B1012912D015E14946B0F5BE7F97
:104DC000FAD92E70CC718C71EC702C72287A0A187A
:104DD000401CC0B2147228720F28F7D303E1B9F84F
:104DE00002204946824201D9EE7100E0EC719148FF
:104DF0008A7908300F2A15D2CB79082B0BD2C3F150
:104E00000708EB7912F800C003FA08F3634413545F
:104E1000CA79521CCA71CA79082A03D18A79521CEC
:104E20008A71CC7199F80610C8460F2973D10D21EB
:104E3000FCF782F8A881010A6970C0B2A87088F8EE
:104E4000064098F816208A4265D198F815108142DC
:104E500061D198F80BC07949032302227848BCF14C
:104E6000000F10D0BCF1010F02D0BCF1020F14D022
:104E700080F86A2000E0C9E091F800C02CF00C0C2A
:104E80000CF1080C0FE080F86A6091F800C02CF07B
:104E90000C0C0CF1040C06E0A7E080F86A3091F8E5
:104EA00000C04CF00C0C81F800C098F80C10B6EB68
:104EB000111F04D180F86E4087F846400EE0B2EB37
:104EC000111F04D180F86E6087F8466006E0B3EBEE
:104ED000111F03D180F86E2087F846200B0717D0EA
:104EE00001F00F01012901D0022915D080F86C6072
:104EF0002C7198F80D102A7906FA02F30B406B71A9
:104F0000082A41D2DFE802F00B0F4016212C333A79
:104F100080F86C40ECE766E080F86C20E8E713B3BB
:104F200080F8704030E013B180F850602CE080F8D9
:104F3000504029E023B180F8656087F8036123E0E1
:104F400080F8654087F803411EE023B187F8F540FB
:104F500080F84D4018E087F8F56080F84D6013E068
:104F600013B180F868600FE080F868400CE013B17E
:104F700080F8666008E080F8664005E013B180F8CC
:104F8000676001E080F86740521CD2B22A71082A9B
:104F9000B1D398F80E102B4A8B0705D587F8F1602E
:104FA00080F86460568104E087F8F14080F864403E
:104FB0005481C90702D080F8294001E080F82960B7
:104FC00098F8111000F86D1FC2781F48012A1FD0F1
:104FD00009B3012922D04FF4805100BFA0F8761008
:104FE0001A493C200870A9F80240A9F80440B9F811
:104FF0000210491CA9F80210B9F80210B1F5FA7FA5
:1050000004D940F2F511A9F802102C70BDE8F08324
:1050100044F21C71E2E74FF40051DFE741F25551D1
:10502000DCE7000023070020AC020020480100203C
:1050300000100140A80C0020BC060020D004002075
:10504000C00C0020600A0020380500202007002046
:105050002DE9F05FFDF748F98E4D2888A5F104068B
:10506000C0070AD0308820F008003080288820F05F
:105070000900288001F042FED9E02888DFF8189264
:10508000DFF81882864C80071AD5B9F8001041F075
:105090000101A9F80010B8F800008049143150301F
:1050A000088028884FF6F95108402880308840F061
:1050B00004003080FEF75AFF84F83C00BDE8F09F02
:1050C0002888784F4007288871D520F00400288070
:1050D000FEF74CFF94F83C108142EFD1308820F06D
:1050E00004003080FDF7D8FA2078410605D594F801
:1050F000541094F83B209142E0D03978400621F0DA
:105100000201397004D5FEF70DFA97F82F7004E00C
:1051100094F83C00FDF73AF90746DFF880B140F615
:105120008C2A0BF1180B062F47D294F83800B8429E
:105130003ED03846FDF7AEF82078C00716D094F878
:105140003A0094F8391000F00302914206D0A17A97
:1051500000F0010001F00101884215D1FDF704FAC9
:10516000FBF74CFEFDF72CFB384689E0FDF7FCF918
:10517000FBF744FEFDF724FB3846FDF715FA2078CF
:1051800040F00100207099E7288820F0080028806E
:10519000206B810801EBD000504515D2B8F8001003
:1051A0000844ABF80000308840F0080003E00DE050
:1051B000308820F00800308080E7B9F8001041F016
:1051C0000101A9F80010DFE75046E7E7000728884B
:1051D00031D520F008002880308820F00800308089
:1051E000FEF7C4FE84F83C00FDF756FA387820F04C
:1051F000020038702078400604D5FEF793F997F83E
:105200002F5004E094F83C00FDF7C0F80546062D49
:1052100008D294F83800A842B5D0FDF7A5F9FBF7FD
:10522000EDFD2AE02048C18841F04001C180BDE881
:10523000F05FFDF7A5BAC006288825D520F010003C
:105240002880308820F01000308097F838000C2833
:1052500002D2401C87F83800387840F002003870DD
:10526000FEF760F997F82F50787884F8390094F8B1
:105270003800A84287D0FDF777F9FDF7A1FA284654
:10528000BDE8F05FFDF790B94EF2BE1108402880EE
:1052900014E7000010040040000400402404004013
:1052A0004801002058040020600A00202DE9F04F3A
:1052B000514F85B0388820F0010038804E480026D4
:1052C000103006804D4CDFF838A14FF0010894F8FB
:1052D0005C0042F63029C10774D072B64948816932
:1052E00041F400718161816941F4806181614FF411
:1052F0000040FEF7A1FD444D00212846FBF7DCFAF3
:1053000000212846FBF7CEFADFF800B1002158460D
:10531000FBF7C8FA00213E48FCF732F92846FBF7B4
:10532000E7FB5846FBF7E4FB4FF46020CDE90206AB
:105330008DF8056000968DF810808DF80480694620
:105340002846FBF767FC01231A460F212846FBF786
:10535000B2FC01212846FBF7A5FA00204946401C73
:1053600080B28842FBD328462E600121FBF7E2FC85
:1053700028688007FCD524484C30006894F85C10FD
:1053800021F001012144A1F85000FBF79FFA62B619
:10539000FDF7D4FF47F69061AAF8001094F85C007E
:1053A000401CC0B284F85C000C2822D2124914318F
:1053B000A1F80080388840F00100388005B0BDE8D1
:1053C000F08FFFE7134920F00100085A12490880C6
:1053D000114945F65800083908800F4847F258012E
:1053E000001F01800C4920200C390880AAF8009089
:1053F000D4E70320A070E1E7000800405804002033
:105400002C08004000100240002401400028014008
:1054100008000240F88E0008202C01400029018875
:1054200002D041F0800101E021F08001018070474D
:1054300010B50A884B88CC881A438B8823431A43BB
:105440000B891A434B8989891A430A43A0F84420DF
:1054500010BD0021018041808180C1800181418196
:10546000818170470029818802D041F0010101E06B
:1054700021F00101818070470029018802D041F0AC
:10548000010101E021F0010101807047002930F89D
:10549000441F02D041F4004101E0C1F30E0101803C
:1054A000704700004B4910B5884202D10121C41455
:1054B00086E0B0F1804F09D0474988420DD10121E3
:1054C0000220FEF7DBFC0021022064E001210846F7
:1054D000FEF7D4FC002101205DE04049884206D15E
:1054E00001210420FEF7CAFC0021042053E03C49BE
:1054F000884206D101210820FEF7C0FC00210820C7
:1055000049E03849884206D101211020FEF7B6FC57
:10551000002110203FE03449884206D1012120209B
:10552000FEF7ACFC0021202035E03049884202D152
:105530000121441444E02E49884202D10121CC04C7
:105540003EE02C49884202D101210C0538E02A496D
:10555000884202D101214C0532E02849884206D117
:1055600001214020FEF78AFC0021402013E024495D
:10557000884206D101218020FEF780FC0021802096
:1055800009E0204988420AD1841501212046FEF70E
:1055900075FC00212046BDE81040FEF76FBC1A499B
:1055A000884202D101210C040AE01849884202D144
:1055B00001214C0404E0164988420AD101218C04DF
:1055C0002046FEF773FC2046BDE810400021FEF7A0
:1055D0006DBC10BD002C01400004004000080040DC
:1055E000000C004000100040001400400034014056
:1055F000004C0140005001400054014000180040A0
:10560000001C0040002000400040014000440140D8
:1056100000480140002A828901D00A4300E08A4301
:105620008281704730B5028C22F001020284028C24
:105630008388048B22F0020224F073050C882C432B
:105640000D8915434A882A43114DA8420BD0114DAC
:10565000A84208D0104DA84205D0104DA84202D053
:105660000F4DA8420DD122F008054A8923F440735A
:105670002A4322F004058A882A438D891D43CB8959
:105680002B4383800483C9888186028430BD000057
:10569000002C014000340140004001400044014022
:1056A00000480140028B22F008020A43028370473F
:1056B00070B5028C22F010020284028C8488038B65
:1056C0000D8823F4E6464FF6FF7303EA05253543BC
:1056D0000E8922F0200203EA061616434A8803EADE
:1056E00002123243104EB04202D0104EB04215D1D9
:1056F00022F080064A8924F4406403EA021232430D
:1057000022F040068A8803EA021232438E8903EAB5
:1057100086062643CC8903EA8404344384800583C7
:10572000C9880187028470BD002C0140003401400B
:10573000028B4FF6FF7322F4006203EA012111434A
:105740000183704770B5028C22F480720284028C4F
:105750008488838B0D8823F073031D4322F4007328
:105760000E894FF6FF7202EA06261E434B8802EAB4
:1057700003233343104EB04202D0104EB04215D135
:1057800023F400664B8924F4405402EA0323334394
:1057900023F480668B8802EA032333438E8902EA6E
:1057A00006162643CC8902EA041434438480858398
:1057B000C9888187038470BD002C014000340140FA
:1057C000828B22F008020A438283704770B5028CF4
:1057D00022F480520284048C8288838B0D8823F407
:1057E000E6464FF6FF7303EA0525354324F40056D9
:1057F0000C8903EA043434434E8803EA0636264310
:10580000094CA04202D0094CA04205D122F48044A8
:105810008A8903EA8212224382808583C988A0F89C
:105820004010068470BD0000002C0140003401408F
:10583000828B4FF6FF7322F4006203EA01211143C9
:1058400081837047018582827047828822F07002CE
:10585000828082880A4382807047A0F84010704797
:1058600030B502881B4B1C4C98420DD0A0420BD087
:10587000B0F1804F08D0194DA84205D0184DA8426C
:1058800002D0184DA84203D122F070054A882A435D
:10589000154DA84206D0154DA84203D022F44075FC
:1058A000CA882A4302808A8882850A8802859842AB
:1058B0000AD0A04208D00E4A904205D00D4A90422C
:1058C00002D00D4A904201D1097A018601218182DC
:1058D00030BD0000002C01400034014000040040B5
:1058E00000080040000C0040001000400014004080
:1058F0000040014000440140004801404FF6FF7164
:10590000818000210180C18041800172704700299F
:10591000018802D041F0020101E021F00201018082
:1059200070470029018802D041F0040101E021F014
:10593000040101807047000030B52348244B90F8E3
:105940002010026801F01F00204951F82000024297
:10595000186802D040F4803001E020F480301860F4
:105960001C484FF00005807941061B482AD41B498A
:1059700002880C88A21A92B201240F2A12D30A8834
:1059800002808268002A00DA5242062A0ADD144A9E
:105990001278022A06D193F80D2102B94477C5770F
:1059A0000A884280427F012A02D00988418030BDA6
:1059B00042880988891A89B240F21A629142F6D364
:1059C000C47730BD457730BDE80500203C93000822
:1059D000AC020020600A0020880C00202C07002068
:1059E000230700202DE9F0414D6800231E240F22DB
:1059F000854202DD0868BDE8F081D1F8F4508542A7
:105A000002DAD1F8F000F6E701EBC2056D688542D5
:105A100001DA134600E01446E21852085D1CAA425F
:105A2000F2D101EBC20351F832505C68844202DAD1
:105A3000D3E9026701E053E90267001BC11789053A
:105A40003A1B41EA9021D3178005FAF76BFB721BD2
:105A5000A0FB024601FB0261D31700FB0310810289
:105A600041EA94502844C6E72DE9F04FDFF8B8B179
:105A70006A48DFF8AC91DFF8ACA190F80EC0BBF932
:105A80001A70BBF91C60BBF91850BBF96C10BCF163
:105A9000070F48D2DFE80CF08D041A30485E76001C
:105AA000D9F800208284DAF80020C284828CC38C6A
:105AB000A7EB820212B2A6EB83034A431BB25943FF
:105AC00042F3CF2241F3CF23D11870E0D9F8002060
:105AD0004284DAF80020C284428CA5EB820213B221
:105AE000C28C4B43A6EB820212B243F3CF24514344
:105AF00041F3CF23E11814E0D9F80020C284DAF88A
:105B000000204284C28C438CA6EB820212B2A5EB29
:105B100083031CB24A43614342F3CF2341F3CF24B2
:105B2000191949420AB244E0D9F800208284DAF80F
:105B300000204284828C438CA7EB820212B2A5EB38
:105B400083034A431BB2594342F3CF2241F3CF248C
:105B5000111914E0D9F800204284DAF80020828478
:105B6000428C838CA5EB820212B2A7EB83034A43DB
:105B70001BB242F3CF24594341F3CF22A11849422B
:105B80000BB216E0D9F80020C284DAF80020828433
:105B9000C28C838CA6EB820212B2A7EB83031CB2E9
:105BA0004A4342F3CF23614341F3CF22991849423C
:105BB0000CB2BBF91E50594605F21E56A64201DA38
:105BC000CE8306E0A5F21E55A54201DDCD8300E09F
:105BD000CC83B1F9204004F21E55954201DA0D84C0
:105BE00006E0A4F21E54944201DD0C8400E00A8415
:105BF000B1F9222002F21E549C4202DAABF8224094
:105C000008E0A2F21E529A4202DDABF8222001E027
:105C1000ABF82230417B8173BDE8F08FAC020020ED
:105C20003C2401403C280140380500202DE9F04784
:105C300004466D486E4E002702786C48022AB0F97F
:105C4000301004D0082A7BD0092A7AD0C8E0C27B61
:105C5000022A02D1B0F8402052B1A4F8421071815A
:105C60000423B6F908101A460020FEF703FFAEE041
:105C70006049DFF88481496A0D14E580806841023B
:105C800016D5B4F9020040F2DA21884248DD40F22C
:105C90006A41884205DD00BF0823B4F942101A4664
:105CA00060E0A0F2DA20FAF7B8FB0022534B68E07C
:105CB000C0F3C001C0F30020DFF8449181420CD151
:105CC000D8F8440040F2BA4188426DDD40F66A11CE
:105CD0008842E1DCA0F2BA404FE04A480078C006B2
:105CE0000CD5D8F8440041F2243188425CDD41F201
:105CF000D4718842D0DC00F6DC401EE04248DFF878
:105D00000C9190F8701001290BD090F86F000128C9
:105D100007D03F480178C90746D03E49098889B174
:105D200042E0B4F9020041F6DC6188423CDD42F217
:105D30003411884212DC00F59270A0F500501CE08E
:105D400047E04BE0B0F91000B4F90210A0F59672EC
:105D5000914229DD00F5967291420BDDB4F94210B3
:105D600020231A460020FEF785FEA4F842000028F2
:105D700017DB1BE0081A00F59670FAF74EFB0022BD
:105D80004B46FAF7B6FA0E22FAF722FBFAF77CFB3B
:105D900000B2C0F5804068438013A4F84200002D93
:105DA00004DCA4F8427001E0A4F84250B4F84210B8
:105DB0001948F180D8F844304364A0F84C10B0F88A
:105DC0004E10718198F80A10008F01B9404230815D
:105DD00006E01248B0F87C00708100E071813781E4
:105DE00084F84070BDE8F08723070020AC02002053
:105DF00064000020380500204801002000007940A0
:105E000000C0924004070020C00C002000C0824067
:105E10005009002020000020FC080020740A002007
:105E20002DE9F041B1F9025000232B2415228542BF
:105E300003DAB1F90000BDE8F081B1F9AE50854256
:105E400002DDB1F9AC00F6E701EB8205B5F90250CD
:105E5000854201DD134600E01446E21852085D1C3D
:105E6000AA42F1D101EB8205B5F90230834206DA8C
:105E700035F9026C35F9044C31F9221006E01E4662
:105E800031F92240B5F90630B5F90410801B091B21
:105E9000C5178911AD0345EA90458703A1FB070C9F
:105EA000CA1702FB07C201FB05219A1BD317FAF799
:105EB00039F9000A40EA0160001900B2B0F5804FDC
:105EC000B9DB43F6FF70B6E770B5134C40F22445DA
:105ED0002946204600F03EF800281BD0204600F05E
:105EE000C7F82946204600F01DF80C4C002120463A
:105EF000FBF746FB2046FBF7C1FBC0F164000849F5
:105F0000C0B20428087201D900F046F9BDE870401B
:105F1000FBF7FABB70BD000000380140580002409A
:105F2000740600200A0A01219140C943018070478C
:105F30000029818902D041F4005101E021F400518F
:105F400081817047002A828A01D00A4300E08A4397
:105F50008282704730B501F01F0201240025C1F391
:105F6000421304FA02F2012B0FD0022B0FD0838AC6
:105F70004FEA11210088134204FA01F400EA0400F8
:105F800001D000B10125284630BD8389F0E7038A9E
:105F9000EEE710B5C1F3421301F01F040121A14047
:105FA000012B07D0022B07D01430002A026805D03D
:105FB0000A4304E00C30F8E71030F6E78A43026049
:105FC00010BD000030B50446008A85B00D464CF681
:105FD000FF710840E98801432182A1894EF6F31040
:105FE0000140A8882A8910436A890A431043A08186
:105FF000A08A4FF6FF410840A9890143A182684663
:10600000FDF760FF1948844201D1039800E002982F
:10601000A189090400EBC00101EB0010296801D53A
:10602000490000E08900B0FBF1F06422B0FBF2F11E
:1060300009010B096FF018056B4300EB8300A3897E
:106040001D044FF0320306D503EBC000B0FBF2F0A5
:1060500000F0070005E003EB0010B0FBF2F000F0E9
:106060000F000843208105B030BD0000003801401A
:106070008088C0F308007047F8B501210920FDF7BA
:1060800009FF01218803FDF705FF10258DF8035056
:106090002020ADF800001A4E03248DF80240694616
:1060A0003046FCF769F816490C31086820F02000EA
:1060B000086018208DF803004020ADF800008DF82E
:1060C000024069463046FCF757F848208DF8030037
:1060D0008020ADF8000069463046FCF74DF88DF899
:1060E00003502801ADF800008DF8024069463046A3
:1060F000FCF742F801210420FCF790F8F8BD0000FD
:10610000000C014030B585B0FFF7B6FF00244FF416
:10611000E1300090ADF808400C201D4DADF8044072
:10612000ADF80A00ADF80640ADF80C4069462846C7
:10613000FFF748FF25208DF8100004208DF811008E
:106140008DF8124001208DF8130004A8FDF786FB9E
:10615000012240F224412846FFF71BFF0121284677
:10616000FFF7E6FEFBF7FAFA012280212846FFF747
:10617000E9FE012240212846FFF7E4FE0122022128
:106180000448FBF78FFAFBF7E9FA05B030BD0000D1
:10619000003801404400024070B51D4D00242878AD
:1061A000432834D16878462831D1A878502807D0C0
:1061B000512805D0812803D0892801D0212826D153
:1061C000144E7071E9787172A81C891CFAF7ECFE04
:1061D000B072717A294409793182884217D106F167
:1061E0000E00017841F0020101700B48016841F096
:1061F00020010160317A0948002204E02B5D03553B
:106200002A55641CE4B28C42F8D38078707170BD5A
:10621000BC070020740600200C0C0140F20B00208B
:1062200070B51D20FDF7F9FAFDF77CF91D20FDF78B
:106230000AFB154890F82F10144D0623144C85F8CE
:10624000381090F83B1095F83B201143012A04D0F8
:10625000022A07D0042A0AD010E0827A8A420DD09E
:10626000007B09E0027D8A4208D0807D04E0827FC5
:106270008A4203D090F82000884200D12370002089
:1062800085F8400070BD000058040020480100203F
:10629000230700200B4800214180A0F1B8018A8922
:1062A0008280CB891A44C2800B8A1A4402814B8AAD
:1062B0001A444281898A1144818143F6FF71C18168
:1062C0007047000000020020084940F61C72B1F936
:1062D0000C00904202DA00F59F7005E041F2E30203
:1062E000904201DDA0F59F70C881704764000020D6
:1062F00038B51348C16941F00401C1611E208DF811
:10630000000002208DF801008DF8020001248DF8B4
:1063100003406846FDF7A2FA0A498420088009492B
:1063200047F690602C3108800020091F088005493D
:1063300014310C80091F0880081F048038BD00003C
:10634000001002400008004030B420491E4A457841
:106350008B7A114692F83B4091F83910AC4218D133
:106360004BB10379994202D04379994201D14079E6
:106370001AE0807909E08379994202D0C479A14278
:1063800002D182F82F3011E0407982F82F0030BC22
:106390007047C578AC42FAD16BB1C379994202D04B
:1063A000037A994205D1007A82F82F0030BCFEF7BB
:1063B00003BC407AE9E7437A9942E2D00479A142EA
:1063C000DFD0007AE1E700005804002048010020F7
:1063D000FEE700002DE9F0470446007F012868D160
:1063E0003548E1880288511A89B2072916D30088F6
:1063F000E080B4F9000044F2DD414843401346F622
:10640000D96148438013A060401000B2A0814FF0D2
:106410008051B1FBF0F0F9F7FBFF2061B4F90C609B
:1064200096B1B4F902104DF6B05048430014A08262
:10643000B4F904704DF6B05207FB02F24FEA224560
:10644000E58204D4024603E00020E08330E04242CB
:1064500012B22283002D01DB2B4600E06B421BB2FF
:10646000DFF85890638398464FF4804AB24208DAC6
:10647000F9F7C5FF2169F9F798FEF9F7ECFF8013EA
:1064800004E0002901DA484600E05046E083B045C8
:1064900009DA2846F9F7B3FF2169F9F786FEF9F71B
:1064A000DAFF801304E0002F01DA484600E050468E
:1064B0002084BDE8F08700002C07002000C0FFFF0B
:1064C00070B53B483B4D3C4C0078022805D1E87B39
:1064D000022802D1B5F8400028B1288EA4F84E0059
:1064E0000020208770BD3448324995F80D21B0F85E
:1064F000440091F8461000B240F6AA262AB119B31A
:10650000012928D0022933D03CE0E9B12B49097890
:10651000C1F3810101290CD002290DD02849FBF7D4
:1065200083FC80B2A4F8400095F84610012906D0FB
:1065300028E02349D83909E021496C3906E0B04206
:1065400020D340F6F41003E01D496C31FBF76CFCDE
:10655000A4F8400016E01A49FBF766FC80B240F64A
:106560003E11A4F8400088420CD3A4F8401009E082
:106570001349FBF759FC80B2A4F84000B04201D3A4
:10658000A4F840600C49B4F840004831383401F0B8
:1065900083FAB4F91400B4F912204142514389132B
:1065A0002180B4F9101048438013E08270BD0000D0
:1065B00023070020AC020020FC080020D0040020AB
:1065C000208D00080348002180F82A10C18301872C
:1065D00070470000FC08002010B504000B462D4A4F
:1065E000C3F1000028D56442002B12DAA04207DA7A
:1065F000214600F02DFA32F81000C0F5404041E08D
:106600000146204600F024FA32F8100000F5004060
:1066100038E0A34208DA2146184600F019FA32F8A9
:10662000100000F540402DE0204600F011FA32F84D
:106630001000C0F5803025E0002B12DAA04207DA06
:10664000214600F005FA32F8100000F5804019E00C
:106650000146204600F0FCF932F81000C0F5004079
:1066600010E0A34208DA2146184600F0F1F932F8AA
:106670001000C0F5804005E053B1204600F0E8F975
:1066800032F81000B0F5004F01DDA0F5803010BDEC
:10669000002010BD048F000840438013494300EBE5
:1066A000A13000220302002B14DDB3F5001F01DC32
:1066B000802001E04FF4005093FBF0F1014401EB26
:1066C000D1714910814206D0521CD2B20846062A26
:1066D000F2D300E00021C80000B2704702E008C811
:1066E000121F08C1002AFAD170477047002001E04C
:1066F00001C1121F002AFBD1704700002DE9F047AD
:10670000A74CA84821880288511A89B20F297DD345
:106710000088A4F13C052080288F08B1401E2887FE
:1067200095F800C0A04ACCF3810001281DD00228B2
:1067300020D0D18B9D4E9A48DFF87492F388407E2A
:106740000027B1F5926F1CD8142818D378206076F2
:1067500043F01000F08040F26660A8812CF0010048
:106760002870D77389F8007018E0D08B00EB4000D8
:10677000C00302E0D08B8F494843010CDAE7401C8C
:1067800004E0B1F5DB6F09D310B1401E607605E07F
:1067900023F01000F0804CF001002870B5F90200E1
:1067A000B5F914304143C3EBC303C1F38F31C3F3D5
:1067B000D10303EB510109B2A9829046D28B4FF06D
:1067C00080535043B5F91620C0F38F30C2EBC2029C
:1067D000C2F3D10202EB500000B2E882AA6A42433F
:1067E0001213EA6293FBF2F22A63734A1080A268E2
:1067F0000A44A260E1680144E160207C401CC0B210
:106800002074072802D942F3CF0000E0C5E02883B6
:10681000C9106983E760A76041F6C8012774884200
:1068200004DD298B654AB2FBF1F1E981C1178903C7
:1068300041EA9041800342F69B420023F9F772FC43
:10684000A88457485E49A0F13C002A78B0F90600B8
:106850005FEA827C00FB01F14FEA2143C2F3810130
:1068600015D5012907D002290BD04FF268514143B9
:106870000914A18011E049F68C4148430014A0801E
:1068800020E04CF6183141430914A18026E001298B
:106890000ED0022918D0A0806B844A4948430014C6
:1068A000A4F81E00FBF7E0F847480088C0B143E0B9
:1068B0004AF65C3141430914A1804BF62C21484330
:1068C00000146884E383EDE74DF2AC5141430914B1
:1068D000A1804EF27C414143091469843B49DDE7C4
:1068E00095F8200000BB88F80F7089F80070B5F9A2
:1068F0001A00A0F50C519F39B1F56E7F18D8617F51
:10690000F42912D93249E8802E4AA1F846005043B2
:106910000014A880A1F84400FF2085F8200081F829
:1069200028002C493C20087006E0491C617703E0F0
:10693000607F08B1401E6077B5F91A10B4F91E00E7
:1069400081420EDDA07E7D2809D9F08840F0080044
:10695000F0802148017821F0020101700EE0401C16
:1069600006E0A0F23D10814208DAA07E10B1401E80
:10697000A07603E0F08820F00800F080B5F9181048
:10698000606908446061217E491CC9B221761F29D3
:1069900003D94011A88367612776BDE8F08700001E
:1069A0000C0500202C070020AC020020600A00200B
:1069B0002307002030330100140A002074E8260B5E
:1069C000CC0E0100488501002E070020D0450100B3
:1069D000C00C002020070020E2050020024941F6FB
:1069E0008B30886270470000D004002070B5164CD0
:1069F00006252078062825D2DFE800F003080E14CB
:106A00001A211248FAF70EFB012016E00F48801DEC
:106A1000FAF708FB022010E00C480C30FAF702FBF2
:106A200003200AE009481230FAF7FCFA042004E0D7
:106A300006481830FAF7F6FA0520207070BDFAF70C
:106A400011FB2570257070BD24070020F88D00080B
:106A5000090A05D0B0FBF1F0FF2800D9FF207047EC
:106A600000207047D0E90021C368521A5A4301EB55
:106A7000A231816041607047B0F90020B0F9021086
:106A8000B0F90630521A5A4301EBA231818041809D
:106A90007047000030B5494B188849490A8A801A66
:106AA00085B24848484A0F2D047801F150001DD3A3
:106AB0001D880D82117A090713D5022C01D0434994
:106AC00012E0434DB0F90210B5F90050A94205DCBF
:106AD00002DA01F1020108E0458007E0A1F10201BC
:106AE00003E0022C02D13B4909884180B0F84010F4
:106AF0001D88691A89B29C2949D31988A0F84010C9
:106B0000916A0023B1F5804F31DB3349096DB1F54E
:106B1000405F2CDD314940F26665B1F91010A942A1
:106B200012DD43F69915A94202DB40F2333108E049
:106B300040F23335A1F26661694343F2333591FB8C
:106B4000F5F1A0F8441001E0A0F844302449B2F86F
:106B500006510978C1F381012DB100BFB0F844108E
:106B600001F21E511CE092F84620022A10D0A0F833
:106B70004430022C01D0A0F84430B0F95C10B0F9D8
:106B8000443001F114029A420DDAA0F85C2030BDC5
:106B9000012901D00229E1D1B0F8441001F23331CA
:106BA000A0F84410E5E703F11402914203DD143923
:106BB000A0F85C1030BDA0F85C3030BD2C07002080
:106BC0001400002023070020AC020020CE04002087
:106BD000CC040020C8040020480100203805002013
:106BE000D00400202DE9FC4101210220FDF73AF9F3
:106BF00001211920FDF74EF901213C48FBF70EFB5E
:106C00004027ADF8007003248DF802400420384D71
:106C10008DF8030069462846FBF7AEFAE001ADF8AF
:106C200000008DF802401C208DF8030069462846BC
:106C3000FBF7A2FA4FF4E0712846FBF724FBA815F6
:106C4000ADF800008DF8024010208DF80300694671
:106C50002848FBF791FA4FF4A060FCF731FE1D20A5
:106C60008DF8040001268DF8056000258DF806508A
:106C70008DF8076001A8FCF7F1FD1F498C20088002
:106C80001D494FF6FA702C3108806E20091F0880CC
:106C900019481430068018480830078016492031FA
:106CA0000D80154AD020121D1080134A45F2F300C2
:106CB000183210800A1F45F2500010800E4A4FF61D
:106CC000FF7038321080121D1080121D108041F2AA
:106CD0001B10088000F012F8FBF752FD0648103038
:106CE0000580001F0480BDE8FC810000000C1A0034
:106CF00000100140000C01400004004070B51D2050
:106D0000FCF780FD2A4D40212846FBF7B3FA8400AA
:106D100080212846FBF7AEFA44EA4004A91528462C
:106D2000FBF7A8FA0443E0B2224C84F83C00FBF7DE
:106D30002DFB0546052805D91F48C18841F04001B3
:106D4000C18001E084F838501C48007A000703D560
:106D500094F838001A490D5C4FF6FA702063E0622F
:106D6000A06260622062E061A0611648606300205A
:106D70006064206584F83F0084F84000FBF7B4FAB3
:106D8000A07AFF2811D0022084F83D000E48008828
:106D9000A0662846FBF756FF207820F001002070FF
:106DA000BDE870401D20FCF743BD0120ECE700006A
:106DB0000010014048010020600A0020AC020020C1
:106DC00000980008DCFF0500240400402DE9F04392
:106DD0004E484F4902880B889A1A92B20F2A69D3FB
:106DE000098801804B49098B027D00EB42029180AA
:106DF000017D491CC9B2017508295BD300240475C3
:106E00002246017D00EB4103491CB3F90430C9B2AD
:106E100002EB630212B201750829F2D33E490475F0
:106E20003E4B4A8044800E789D895FEAC67C40F6DE
:106E300038694FF0030714D0A2F22B5C42F6E858F1
:106E4000C44520D3A1F1020C26F00204ACF80020C6
:106E500047750C7040F22B54A24211DA45F004023F
:106E60001EE046F001060E704A4507DD45F00102BE
:106E70009A8126F002020A70477519E0447517E0FE
:106E800045F002020CE04A450CDA8775427D12B1EA
:106E9000521E42750CE046F002020A7025F007020D
:106EA0009A8105E0B30703D5837D2BB15B1E837503
:106EB00040888880BDE8F08342F6AA239A4222DA0D
:106EC000B1F904302BB941F2CD05AA4201DA448070
:106ED000EEE7134C920302EB843241F67244B2FBAC
:106EE000F4F214B240F2333502464480AC4200DA88
:106EF0005580B2F90240E41A04F5A374B4F5237F77
:106F0000D6D84380D4E74FF48043FAE7F40A002050
:106F10002C070020AC020020E2050020600A0020BF
:106F2000C8F1FFFF2DE9F0416D4CDFF8B8E14FF0FB
:106F3000000594F83410C80706D094F938104B4275
:106F4000002958DD0E4657E0674884F83750A4F80A
:106F50004250664A90F8380084F840001586CEF812
:106F60000450CEF80850624E40F26663CEF80C50E2
:106F7000A4F87C3036F810005E4E768830444FF628
:106F8000FF7606EA800024F8300B4FF0806044F86A
:106F9000040CA320208460845810A084E38440F66D
:106FA00099102085580060854FF48050A08541F2EB
:106FB0003330E08541F26660208641F699106086A4
:106FC00041F6CC40A0864FF40050E08642F23330C8
:106FD000208742F26660608742F69910A08742F6E9
:106FE000CC40E08782F89D5041F00100207184F888
:106FF0004450BDE8F0811E4694F937004242002813
:1070000001DD074600E01746F61B012E0BD00028D5
:1070100000DB02465FFA82F684F8380094F84F00ED
:10702000012805D041E0002900DA1946CEB2F3E785
:1070300094F939305942002B01DB184600E008462C
:1070400094F93A20C7B25042002A01DB944600E08E
:107050008446BC4508DD002A00DA0246D7B2002B80
:1070600000DA0B46D8B207E0002B00DA0B46DFB29D
:10707000002A00DB1046C0B204EB4000B0F950100B
:1070800004EB470030F9502F11444910018084F877
:107090004F5084F83E5084F83D5084F83C5084F8BA
:1070A0003B5084F83A5084F8395004EB460075465A
:1070B000B0F9500024F8420FBEF80410C82309B2FA
:1070C0006422FDF7D7FC6860E968401AA9680844A3
:1070D000A860B5F900104843C013E860608788E7EE
:1070E000740A0020D005002048010020AC020020D6
:1070F0001298000864000020F0B4544890F834104E
:10710000C90776D0524990F84030002291F83810E3
:107110008B426FD04F4CA0F872204F4DE65C044676
:107120008E4294F9374002D0EE5C8E420FD1641C3F
:1071300064B280F83740EB5C8B4202D1641C80F86B
:10714000374090F937300F2B1BDD0F2317E0434DED
:10715000EE5C434D8E4202D0EE5C8E4211D1641E35
:1071600064B280F83740EB5C8B4202D1641E80F839
:10717000374090F937406FF00E039C4201DA80F8F7
:107180003730324B90F83F50393390F83740EC5459
:1071900090F83F305B1CDBB280F83F30062B01D308
:1071A00080F83F2090F9394090F93B309C420ED155
:1071B00090F93D40A3420AD190F93A4090F93C3011
:1071C0009C4204D190F93E40A34200D1012280F8B4
:1071D0004F201F4A80F8401090F937501378214A09
:1071E000012D0DDD14465E07A46804D544F00804A3
:1071F00003E028E015E024F00804946080F83510DE
:10720000B5F1FF3F0ADA5B07936802D523F0080364
:1072100001E043F00803936080F83510F0BCFBF701
:1072200063B890F84F1001290DD1B0F8721043F6F1
:107230000953491C89B2A0F87210994203D9A0F8E9
:10724000722080F84F20F0BC70470000740A0020C4
:1072500048010020F4970008FA97000806980008F3
:107260000C980008AC02002010B5D0E90021036999
:10727000114481FB03318C0244EA93514260D0E90E
:10728000022382FB0332940244EA93521144816048
:1072900010BD000030B52049204AB1F86A3010888E
:1072A000C01A80B20F2836D31088A1F86A001C4D8E
:1072B00000204FF000432A5C940903D00124B4EB72
:1072C000921F24D1D20622D0164A52F820201268EA
:1072D000134C123434F81040224201EB000494F9AC
:1072E000722008D00A2A04DB0A6823FA00F4224339
:1072F00008E0521C09E012F10A0F05DC0A6823FAC3
:1073000000F4A2430A6002E0521E84F87220401C7E
:10731000C0B21128CFD330BDE80500202C070020D3
:1073200008930008089400082DE9F00779497A4885
:107330000A8903889A1A92B2082A74D300880881AD
:10734000A1F12C0042890AB1521E4281734A92F87F
:107350002820802A67D302F03F020A70C2890AB14E
:10736000521EC281B1F90620902A0CDB8A46FF2A00
:1073700009D08146C089002855D16948002300788A
:10738000092805D005E0BDE8F007624800F09AB989
:107390000823644A92F8EA500DB143F004036248AE
:1073A000817AC90701D043F00203D2F808C05FEA2E
:1073B0000C5101D543F00103176800215B4EFC031B
:1073C00002D596F8654004B18021C4885FEA44681C
:1073D00001D541F040015FEA845801D541F0200118
:1073E0005FEAC47801D041F01001007A400701D56E
:1073F00041F008014E480078C00701D041F0040177
:10740000A00601D541F001010020012D00D1082086
:1074100096F8705085B992F84620022A04D0012AC5
:1074200005D03AB108E072E040F0030004E040F01B
:10743000020001E040F001007A0701D440F0200092
:10744000CCF3C0020025CCF3002C624502D13A07F0
:1074500000D4042596F86F20012A01D145F00105DA
:10746000344A0027BC4612783E46C2F38102012A04
:1074700004D0022A04D0032A04D004E0022602E049
:10748000042600E010262C4A64060ED5214C1C343C
:107490002478240609D51478640606D4274A40F6D1
:1074A000CC44926D6243140C05E0B2F8B62040F66D
:1074B00099146243940B4FF008088AF80A804FF041
:1074C00061088AF80B808AF80C308AF80D108AF867
:1074D0000E008AF80F508AF81070270A4B4083F08C
:1074E0006901414069408AF8117079408AF8124078
:1074F000614052468AF813C071408AF81460517591
:107500004FF4C871A9F80E10FF20AAF80600BDE8D4
:10751000F0077047E80600202C070020E80500204F
:1075200023070020AC020020600A0020C00C0020CD
:1075300050090020D004002048010020200800202D
:107540005048816941F0FC0181614FF4A060FCF773
:10755000B7F9FBF7A3F9FCF717FBF9F721FBFCF7E9
:107560000DF9FDF78DF9FFF73DFBFCF74DF8FFF73F
:10757000C5FBFBF705F9444D4FF40050A5F8160183
:10758000FEF7C0FD00214FF4FA5340F2EE22002036
:10759000401C80B29842FBD3491C89B29142F6D379
:1075A0003A48002680F87260F9F790F9F9F738FE4A
:1075B000FCF71AFBF9F704FDFEF79AFE1022344996
:1075C0003448F8F7E0FD01F0DFF9334C344FE08840
:1075D00020F04000E0803148017821F02001017066
:1075E000FA20F8814FF49670E887FFF7F7F92D49F4
:1075F0002D48FCF776FA2D48FCF798FA2C48416A9A
:1076000088472C48416B8847FEF7DCFF2A48FAF789
:1076100027FA2A494220C8802949C8603E71E0887B
:10762000E0812089208260896082FAF71DFDFAF7E7
:107630007FFCFFF763F801F047F9FFF7C7FB00F0A5
:10764000F9F9FFF727FE01F003F8FEF775F9FAF7ED
:10765000DBFAFBF715FBFFF71DFAFCF701FDFAF764
:1076600037FFFAF769FF00F07BF8FFF75DFE12487D
:10767000FAF7BEF800F06AFAFDF746F9FAF726FACB
:10768000CDE7000000100240AC02002038050020C9
:10769000C00C002028060020600A002048010020BD
:1076A00020070020CC0800209C08002010040020A7
:1076B00038000020E4000020E00900204C070020F2
:1076C00044040020F0B523490278B0F906400023B5
:1076D0001F4E31F81210FF2C18D0B0F904701E4D57
:1076E000BC4231DA00EBE40704F00704BF7AA7409C
:1076F0008478FFB23CB190F801C0ACF1010C644554
:107700001FDA3C061DD455F822200DE056F8222041
:10771000116012498A79521CD2B28A71022A02D3AC
:107720008370C3808B71F0BD11608178491CC9B230
:10773000817042789142F6D38370C188491CC18020
:10774000F0BD56F82220EFE755F822201160F4E74B
:10775000E89400081A93000890940008BC060020E2
:10776000F0B561486149B0F86C200B889A1A92B262
:107770009C2A7BD30988A0F86C105D495D4F91F875
:107780002A1001F0070297F84610022A00D1491E7C
:10779000594C80F83E104FF00203E2884FF0000190
:1077A000550401D5012236E0A489E50601D506225B
:1077B00031E0250701D508222DE0550603D44F4DB1
:1077C0002D78AD0601D5042225E0150501D5072247
:1077D00021E0150601D50A221DE0950601D50C22EF
:1077E00019E0150701D50B2215E0550701D4D50581
:1077F00001D510220FE0D50601D505220BE0650763
:1078000003D4A50701D4E40702D080F86E3007E066
:10781000920403D5032280F86E2001E080F86E10F8
:10782000374A384C92F820E0324A251FD2F808C077
:107830002D4AB2F87060721C92B2BEF1000F0DD0EA
:107840002CF4000CC7F808C090F86E70B7B11E2F6A
:107850001AD090F86F200AB325E007E04CF4000638
:10786000BE60A0F870200A2A01D22360F0BD142A5D
:1078700001D22B60F0BDA0F87010F0BD2B60A0F815
:10788000701080F86F10F0BD642E04D2A0F8702044
:10789000322AEED3E9E7A0F87010EAE77F1C80F8FF
:1078A0006F70A0F8701090F86F20012A10D0002A95
:1078B000E9D0B0F87060761CB6B2A0F870601E2EE9
:1078C000D7D323603C2EDED9521E80F86F20D2E73A
:1078D000B0F87020521C92B2A0F870202360C82A21
:1078E000D1D980F86F10C6E7E80500202C070020EA
:1078F000C00C0020AC020020600A002048010020DB
:10790000D0040020141C0140F0B54248B0F84810E3
:10791000491C89B2A0F8481002297AD33E490024B4
:10792000A0F848400A783D4B042A57D04FF48041D4
:10793000082A0BD0A0F10C02B2F900208A4200DA2A
:107940001146B3F980208A4200DA1146344A92691E
:107950008A4200DA11B2418282881D8AC2EB850216
:10796000304D12B22D78C5F381062A4D42F2917640
:107970007243B5F9765092126A431213C260866858
:107980001546C6EBC60642F3D102F60202EBA6325A
:107990008260C66C1644C664B0F850707F1CBFB2DB
:1079A000A0F85070B7F5806F04D3B6120682A0F825
:1079B0005040C464891A1C4EC26A724340F2555644
:1079C0004E4302EB4602466A32444262B3F930301B
:1079D000B2EB034F06DD1A04426206E01349B1F927
:1079E0000410B3E7002A00DA4462C162104990F83B
:1079F0003D2091F838108A420BD080F83D10B0F845
:107A00004210A0F84410B0F84010A0F84210A0F8BE
:107A10004050F0BD3805002023070020AC020020B4
:107A2000580C0020D0040020C3F5FFFF740C002088
:107A30004801002015481649B0F85A200B889A1AB8
:107A400092B20F2A20D30988A0F85A10B0F900107A
:107A500041F6302251438913A0F86C100D494FF4C0
:107A600080420B78A0F10C01022B06D1B1F9003055
:107A7000934202DA1B1D0B8000E00A800021A0F86F
:107A8000601020F85C1F428070470000380500201D
:107A90002C070020230700204FF6FF7202EA800225
:107AA00010F4404315480ED0B3F5804F14D0B3F511
:107AB000004F4FEA122216D0C2F5807330F813300F
:107AC0005B424B8005E0120A30F812304B80C2F561
:107AD000807230F812000FE0120AC2F5807330F89D
:107AE00013304B8005E030F81230C2F580725B42F3
:107AF0004B8030F812004042088070470491000823
:107B0000104A518A908AD28A16384639A2F1110257
:107B100000D54942002A00DA52421144002800DA16
:107B200040420844084943F6284300B2B1F93620E0
:107B30005A43921340F2D733584302EBA030C88621
:107B400070470000AC02002038050020F0B59049D5
:107B500090480A8903889A1A92B23E2A1ED3008856
:107B6000088101F138004FF4FA63428A9A4202D246
:107B7000521C428200E04382874A92F82220802AE7
:107B80000CD302F03F020A70B1F90620402A06DB4E
:107B9000FF2A04D0C2883AB1521EC280F0BDBDE8AF
:107BA000F0407B48FFF78EBD428A9A42F6D30778B1
:107BB0004FF0010E3A074FF0FF055BD5847A40F293
:107BC000DC52630708D444F004038372C28081F856
:107BD0000BE081F80AE04CE04378072B05D0032B3B
:107BE00003D0052B01D0062B07D1660605D444F03F
:107BF00040038372C280052239E0654A5FEA437C14
:107C000002F138024FF42076127A0DD55FEAC26C89
:107C10000AD45FEA446C07D442F0100202723A06BA
:107C200028D4C680192222E0DF0709D0970707D49D
:107C3000670605D442F002020272C680042216E0F2
:107C40009F0709D5170707D4670605D442F0080235
:107C50000272C68003220AE01B070BD5530709D422
:107C6000630607D442F004020272C6800B22CA7275
:107C70008A72CD80494AB2F92230B2F91A7003F201
:107C80003D140022A74200DB0276414E444C06F12F
:107C90003806A479B6895FEAC46C06F101064FF490
:107CA000C874B6B213D58681B6F57A7F05D9017A44
:107CB00021F0800101728281F0BD037A1E06FBD49F
:107CC000828143F080020272C480112035E09F421D
:107CD00016DA037E052B13D28681B6F5487F04D9C8
:107CE0008281027A22F040020272027A5606E3D4BE
:107CF0005B1C037642F040020272C48002201CE04A
:107D0000284B1C89C4F3C006C4F3002740F2EE24BC
:107D1000BE4216D11E78360713D4427E012ACBD13B
:107D2000428BB2F5167F02D2521C4283F0BD827A9A
:107D300042F002028272C4800F20C8728872CD8025
:107D4000F0BD93F80D714FF40046012F18D1164F76
:107D500041F6583C7F6C674512DD83F80CE1134B0C
:107D60001E60C38AA34202D25B1CC382F0BD4FF4E3
:107D7000FA73C3801C23CB728B72CD80C282F0BD9C
:107D8000C2820A4883F80C21001F0660F0BD000083
:107D9000CC0600202C070020E8050020D00400209D
:107DA000600A0020AC0200204801002014080140B5
:107DB0002DE9F05FFE48FF49DFF8FCA3007E0A1DB5
:107DC000131D012850465AD030F85A4F0C80418874
:107DD0001180BAF85E001880FDF746FEF74DF84CAA
:107DE00049F2CD32B5F91E106183B5F9200043F692
:107DF000CC4C01EB400050430014A083B4F9223076
:107E0000B4F9206000FB03F201FB062242F38F323B
:107E10006282B4F9167007FB0CF7BF1340F2333CD3
:107E2000704302FB0CF201FB130007EBA232E2826B
:107E300040F38F30A082B4F91810E24FC1EBC101BA
:107E400041F3D10101EBE000DF4E2083786C30601C
:107E5000316930468847DD49308948800846FDF75A
:107E6000E5FEDFF86CB301264FF000099BF8000037
:107E700008280CD0618F218204284AD01AE030F8FB
:107E8000604F0C8041881180BAF86400A3E7D148A4
:107E900090F93710491C022939D890F8741019B19B
:107EA000B4F85A00208205E0618F2182A4F85A10AC
:107EB00080F87460B4F91410B4F90A00C64AF9F7EE
:107EC000E9FAE062BAF91611884204DDC248E162BB
:107ED000027C91408162BA48DFF800E3503847F2F3
:107EE000A30802784EF24611002A7AD0012A79D0EE
:107EF00080F800909BF8000004280DD0B64AB4F931
:107F00001210B4F90800303AF9F7C4FA08E0608FAB
:107F1000C8E7686A0014E062B87A002863D0B04805
:107F2000A3462546A062AC4C443C2060E86A6060F1
:107F300020461035FCF76EF8A14928883C39FFF738
:107F4000ABFDDFF87C82A8F15008D8F81410C8F80F
:107F50007010B5F91010A068B5F9122000FB01F7F8
:107F6000E368504303FB127444F38F3703FB0100B3
:107F7000AF8740F38F34EC879A4D28466F80AC80F2
:107F8000FEF728FA287F08F11805012871D0604211
:107F900041104DF6B350474369803A142A80404659
:107FA000A8F804408B18C380891AA8F808108AF82A
:107FB0000C90B8F904305446002B00DD2673B8F954
:107FC0000600002802DD217B891C2173B8F90820F6
:107FD000002A02DD217B091D2173217B072979D22B
:107FE00002E007E02CE05AE0DFE801F07470886EF0
:107FF00084728600B5F91E2042448A420AD8B5F937
:10800000202042448A4205D8B5F9222042448A42BF
:108010007FF670AFA0F80290B7F8B6204946B2F5E7
:10802000C87F01D8467006E0B2F5487F01D8022229
:1080300000E0032242708AF80F108BF8001025E050
:1080400080F80090B5F91EC04A46C4448C4509D852
:10805000B5F920C0C4448C4504D8B5F92250454434
:108060008D42D5D9B7F8B610B1F5C87F02D84670A1
:1080700007E017E0B1F5487F01D8022100E00321B5
:10808000417042808AF80F208BF80020BEF806105D
:1080900041F40061AEF80610F9F73CFF2AE74FF40F
:1080A000AF703DE74F484DF6B352B0F9203059421A
:1080B00049106980B0F91E00504302142A804046DE
:1080C000A8F804306EE705E0667303E0022100E0E3
:1080D000032161739BF80010434E0129434F617BDC
:1080E000DA460DD0072961D2DFE801F060FDFCFB24
:1080F000FAF9F8000421ECE70521EAE70621E8E7B0
:108100000729F0D2DFE801F052042980A5D3F0005E
:1081100001461846FBF7CCFC2860B5F9020040F692
:108120008151484380136880B5F9001040F68152B0
:108130005143891329804218A2F68152B8F80E30B3
:108140005242C3EB620212B2A8F80C20002A01DCF2
:10815000A8F80C90B8F80C206EE1404201B25042F1
:1081600000B2FBF7A5FC2860B5F9020040F681518A
:10817000484380136880B5F9001040F6815251439E
:10818000891329804218A2F68152B8F80E30524263
:10819000C3EB620212B2A8F80C20002A01DCA8F896
:1081A0000C90B8F80C20A4F85E2021E0E9E0000073
:1081B000E0090020342C0140AC02002038050020EA
:1081C0006400002048010020440400200004002036
:1081D00023070020740A0020CC080020600A002039
:1081E000A2FEFFFF140A00200024014000280140E5
:1081F0001044A4F85A00084452E13046F8F72EFD26
:1082000001231A460721B1E019461046FBF750FC3E
:108210002860B5F9020040F6815148438013688018
:10822000B5F9001040F68152514389132980421854
:10823000A2F68152B8F80E305242C3EB620212B27B
:10824000A8F80C20002A01DCA8F80C90B8F80C2043
:108250004DE15942404209B200B2FBF729FC2860C7
:10826000B5F9020040F68151484380136880B5F9A2
:10827000001040F681525143891329804218A2F61A
:108280008152B8F80E305242C3EB620212B2A8F823
:108290000C20002A01DCA8F80C90B8F80C2056E15C
:1082A0003046F8F7DBFC01231A4605215EE0114653
:1082B000FBF7FEFB2860B5F9020040F68151484308
:1082C00080136880B5F9001040F68152514389133C
:1082D0004218A2F681522980524206E076E14AE134
:1082E0001BE1ECE0BCE08FE013E0B8F80E30C3EB2C
:1082F000620212B2A8F80C20002A01DCA8F80C9047
:10830000B8F80C20A4F85C201044A4F85A000844E3
:108310004EE1504201B2584200B2FBF7C9FB28605F
:10832000B5F9020040F68151484380136880B5F9E1
:10833000001040F681525143891329804218A2F659
:108340008152B8F80E305242C3EB620212B2A8F862
:108350000C20002A01DCA8F80C90B8F80C204FE1A2
:108360003046F8F77BFC01231A4606213846F8F719
:1083700075FC01213046F8F7E7FB01213846F8F794
:10838000E3FBB04EBAF8080055463080BAF80A0050
:108390007080BAF81000B0803046F9F775FAB4F87A
:1083A0005A00F1880844A4F86000B4F85C003189F0
:1083B0000844A4F86200B4F85E0071890844A4F887
:1083C0006400317EA048012978D034F85A1F01801A
:1083D00061884180A18881809B49028808310A8098
:1083E00042884A80808888809748896A0830884710
:1083F00095F83E0000287DD0F8F734FE15F83E0FC2
:10840000401E2870BDE8F09F01461846FBF750FB60
:108410002860B5F9020040F6815148438013688016
:10842000B5F9001040F68152514389134218A2F663
:108430008152524229805208A4F85E201044A4F8C8
:108440005C000844A4F85A0000213046F8F77CFB91
:1084500000213846F8F778FB01231A460621CCE6BE
:10846000404201B2504200B2FBF722FB2860B5F94E
:10847000020040F68151484381136980B5F900003C
:1084800040F68152504380130A18A2F6815252429C
:10849000520828801144A4F85E20A4F85A10084419
:1084A000A4F85C0000213046F8F74EFB0021384666
:1084B000F8F74AFB01231A4605219EE6B4E0194667
:1084C0001046FBF7F5FA2860B5F9020040F6815135
:1084D000484380136880B5F9001040F6815251433B
:1084E00089134218A2F68152524229805208A4F8F8
:1084F0005A2000E09BE01044A4F85E000844A4F871
:108500005C0000213046F8F71FFB00213846F8F7E1
:108510001BFB01231A460721C2E65942404209B219
:1085200000B2FBF7C5FA2860B5F9020040F68151A8
:10853000484380136880B5F9001040F681525143DA
:1085400089134218A2F68152524229805208A4F897
:108550005A201044A4F85C000844A4F85E000021EE
:108560003046F8F7F1FA00213846F8F7EDFA012322
:108570001A46062194E61146FBF79AFA2860B5F9E7
:10858000020040F68151484381136980B5F900002B
:1085900040F68152504380130A18A2F6815252428B
:1085A000520828801144A4F85C20A4F85A1008440A
:1085B000A4F85E0000213046F8F7C6FA00213846DC
:1085C000F8F7C2FA01231A460521C9E6504201B262
:1085D000584200B2FBF76CFA2860B5F9020040F689
:1085E0008151484380136880B5F9001040F68152EC
:1085F000514389134218A2F68152524229805208EF
:10860000A4F85C201044A4F85E000844A4F85A00C2
:1086100000213046F8F798FA00213846F8F794FA26
:1086200001231A4607219BE634F8601FCFE607486E
:108630000088A0F5D04168393FF4E4AEBDE8F05FB2
:10864000F9F7B6BBE009002030000020182C0140EB
:108650002DE9F041904C9148B4F862100288511A0B
:1086600089B20F296FD30088A4F862008C48008873
:10867000DFF83082C0074FF000054FF0010741D00E
:10868000874AD4E90C1024321388B1EB530F02D27D
:108690001288511A08444FF4F371884200D20846F8
:1086A0008149B1FBF0F0616CC1F351010844064609
:1086B0006064F7F7B2FE00227C4BF7F71AFE4FF02A
:1086C00040427B4BF7F715FE0E22F7F781FEF7F7D6
:1086D000DBFEA4F8AC0094F86D00401CC0B284F836
:1086E0006D00082834D36C4898F84620001F0378A2
:1086F0009A4201D0027045806E4A13786E4A23B1C7
:10870000458021E06564256558E0D8F89410A1F50E
:10871000FA618E4211DDE16D8B1C9E4205DDB0F9E0
:1087200002100A290DDA491C06E08E4205DAB0F97A
:108730000210002908DD491E4180B0F902000A2814
:1087400002DB177001E0A2E01570E66584F86D5059
:108750005A484FF4A5420178C1F38101012949D05B
:1087600002294AD044F687712181A4F8A820B0F9E3
:10877000243089B24B439B13A4F8A430B0F90E0007
:1087800000237043B0FBF1F0216DC0F3D100C1EBC9
:10879000C101C90200EB91302065F017810341EA65
:1087A0009641B003F7F7BEFCB4F8AA10C1EBC101C3
:1087B000C902C00800EB9130A4F8AA00616C206FD8
:1087C0000844206794F87420521CD2B284F87420B4
:1087D000082A05D3C008A4F8760084F874502567E9
:1087E0003748384EC3885A0633D498F80F20022AE7
:1087F00006D02CE043F20451B6E744F24621B3E739
:10880000B26840F69916B24221DD94F8382094F807
:108810008E60B2420CD084F88E2094F83D2002F095
:108820000106C2F34002964202D1A4F88A5004E045
:10883000B4F88A20B2F5966F05D2B4F88A00401CCD
:10884000A4F88A0005E043F08002C28001E0A4F8A9
:108850008A50114894F83F30B8300C2B01D2C574BF
:1088600000E0C774174A0F4C41F2482692F83C20AA
:10887000B4F8824041F2504C0C2B0AD3B14208DBD1
:10888000012A06D0614502DD002C00D18774BDE8C5
:10889000F0818574FBE70000480100202C070020D0
:1088A00000040040AC0200204564BD0100209C4053
:1088B000133B3340FE030020FF030020D0040020C0
:1088C000600A00203805002070B5284C284821880F
:1088D0000288511A89B23E2947D300882080254852
:1088E000808B254D80022860696928468847234986
:1088F000A868FDF777F822496060CB885A072ED424
:108900000022B0F1F05F0FD9E089B0F5FA7F08D905
:1089100043F00400C8801B48017821F00201017077
:108920001CE0401CE0811AE0B0F1D25F0CD94FF49A
:10893000F031A1EB10308003C910B0FBF1F02061E1
:1089400000280CDA22610AE0B0F1C85F03D94FF4C5
:108950008040206103E023F00400C880E281D4E974
:108960000401884200DB0846A06170BD580C00205D
:108970002C070020AC02002094060020FC96000882
:10898000600A0020E205002005494FF4804048615C
:10899000086188610348C18821F48271C1807047F1
:1089A000580C0020600A00202DE9F041384C394E67
:1089B000394F207841F23331C2074FF000050CD017
:1089C000A28962B394F90700002800DA4042C0B2DD
:1089D000032829D240F2AE702AE0A570E5732F4A31
:1089E000E571A58192F83830237220F00800A1804B
:1089F00040F0020020703D867560B560F560116D35
:108A0000490005D041F68461A18140F0100020703A
:108A1000C0B240F0010020706574BDE8F08165814E
:108A200020F01000207015E0042803D240F6510019
:108A300060810FE0052802D240F69910F8E740F671
:108A4000CC42062803D3072801D3082801D262812B
:108A500000E0618197F89D0098B9B088102301B2B9
:108A6000B4F90A003622FCF705F87060F168401A84
:108A7000B1680844B060B6F900104843C013F06014
:108A80003886388E10B10120A070C6E7A570C4E703
:108A9000740C0020AC060020AC020020480100202D
:108AA0002DE9F041554C2678F0077CD05448217AC6
:108AB000544D90F8380081427BD0534A2346DFF86A
:108AC0004CC1575C93F90E2093F90730874203D0CD
:108AD0001CF80170874213D146F002065B1C267019
:108AE0005BB2E3711CF80110814201D15B1CE371A0
:108AF00094F90710062901DD0621E171521C1CE0E2
:108B0000434F17F801C0434F844503D017F801C005
:108B1000844513D126F002065B1E26705BB2E3711A
:108B2000795C814201D15B1EE37194F907306FF0EB
:108B300005018B4200DAE171521EA273207294F992
:108B400007108A1C042A02D941F68462A2812C4AA9
:108B5000012912780ADD2B4B56079B6802D543F09A
:108B6000080301E023F00803AB606070B1F1FF3F40
:108B700009DA5107A96802D521F0080101E041F0A6
:108B80000801A9606070F9F7AFFBA078012810D147
:108B900021488068A3280CDA94F90700022803DD35
:108BA0000220E07105E01EE06FF00101884200DA6A
:108BB000E171A089002630B1401E0004000CA081A4
:108BC00001D1E671A673E87B04280CD0B5F930100A
:108BD000512341220020FBF74DFF2886002802D1B7
:108BE000E07B10B1A670BDE8F0810C4806700C481F
:108BF0000670207820F001002070F4E7740C00204B
:108C000048010020AC020020F4970008FA97000801
:108C1000069800080C98000838050020400700203E
:108C200023070020743F713D9B3BED396238F436D9
:108C3000A13565343F332A32273133304C2F722E21
:108C4000A32DDF2C242C722B000000361C070038CB
:108C5000AA0A003AAA0A003CCC0C003ECC0C004008
:108C6000380E0042380E0044380E0046380E0048D8
:108C7000380E004AC711004CC711004EC7110050F2
:108C8000C7110052C7110054C7110056C711005830
:108C9000C711005AC711005CC711005EC711006000
:108CA000C7110062C7110064C7110066C7110068D0
:108CB000C711006A00000036220200388E03003A15
:108CC000B005003CD207003EF4090040160C0042FB
:108CD000380E00445B100046C71100483313004AA9
:108CE0009F14004C9F14004E0B1600507717005233
:108CF0007717005477170056771700587717005AE0
:108D00007717005C7717005E7717006077170062AF
:108D10007717006477170066771700687717006A7F
:108D20000000003600000038B600003A6C01003C3C
:108D30002202003ED80200408E0300424404004458
:108D4000FA040046B00500486606004A1C07004CBD
:108D5000D207004E880800503E090052F409005422
:108D6000AA0A0056600B0058160C005ACC0C005C86
:108D7000820D005E380E0060EE0E0062A40F0064EB
:108D80005B10006611110068C711006A0000003412
:108D900000000036000000380000003A0000003CEF
:108DA0000000003E000000400000004200000044BF
:108DB00000000046000000480000004A0000004C8F
:108DC0000000004E0000005000000052000000545F
:108DD00000000056000000580000005A0000005C2F
:108DE0000000005E000000600000006200000064FF
:108DF00000000066000000684414585858701111B3
:108E000058585870411158584870111448585870A3
:108E10001411584858700020007200200070002083
:108E2000006E0020006C0020006A00200068002016
:108E30000066002000640020006200200060002026
:108E4000005E0020005C0020005A00200058002036
:108E50000056002000540020005200200050002046
:108E6000004E0020004CA320004AA32000484721C8
:108E70000046EB210044EB2100428F2200408F226C
:108E8000003E7A24003C7A24003A662600385128B5
:108E900000343D2A0030702D002CA33000287A3495
:108EA000002451380020CC3C001C00400018004039
:108EB0000014004000100040000C0040000800407A
:108EC000000400400000000001020304050005004A
:108ED000010203040104000305020000F001000088
:108EE00036010000F8000000BA0000007C0000001D
:108EF0007C0000007C000000411414111114441186
:108F0000141441110000290052007B00A400CC0081
:108F1000F5001E01470170019901C201EA01130227
:108F20003C0265028E02B602DF02080330035903D9
:108F30008203AA03D303FB0324044C0475049D0499
:108F4000C504EE0416053E0567058F05B705DF0568
:108F500007062F0657067F06A706CE06F6061E074B
:108F600046076D079507BC07E4070B083208590848
:108F70008108A808CF08F6081D0944096A09910963
:108F8000B809DE09050A2B0A520A780A9E0AC40AA1
:108F9000EA0A100B360B5C0B820BA80BCD0BF30B04
:108FA000180C3E0C630C880CAD0CD20CF70C1C0D8D
:108FB000410D650D8A0DAF0DD30DF70D1C0E400E42
:108FC000640E880EAC0ECF0EF30E170F3A0F5E0F25
:108FD000810FA40FC70FEA0F0D103010531075103A
:108FE0009810BA10DD10FF1021114311651187117F
:108FF000A911CA11EC110D122E12501271129212F7
:10900000B312D412F41215133613561376139613A3
:10901000B713D713F6131614361456147514941484
:10902000B414D314F214111530154E156D158C159A
:10903000AA15C815E7150516231641165F167C16E6
:109040009A16B716D516F2160F172C17491766176A
:109050008317A017BC17D917F51711182E184A181F
:10906000661881189D18B918D418F0180B1926190C
:1090700042195D1978199219AD19C819E219FD192B
:10908000171A311A4C1A661A801A991AB31ACD1A7D
:10909000E61A001B191B331B4C1B651B7E1B971B01
:1090A000AF1BC81BE11BF91B121C2A1C421C5A1CBB
:1090B000721C8A1CA21CBA1CD21CE91C011D181DA2
:1090C000301D471D5E1D751D8C1DA31DBA1DD01DB5
:1090D000E71DFD1D141E2A1E401E571E6D1E831EF9
:1090E000981EAE1EC41EDA1EEF1E051F1A1F2F1F6C
:1090F000451F5A1F6F1F841F991FAE1FC21FD71F06
:10910000EC1F002000006400C9002D019201F7014E
:109110005B02C00224038903ED035204B6041A055E
:109120007F05E3054706AB060F077307D7073B0824
:109130009F0802096609C9092D0A900AF30A560B0D
:10914000B90B1C0C7F0CE20C440DA60D090E6B0E26
:10915000CD0E2F0F900FF20F5310B4101511761182
:10916000D71138129812F8125813B813181477142C
:10917000D61435159415F3155116B0160E176B1736
:10918000C91726188318E0183D199919F519511AAD
:10919000AD1A081B631BBE1B181C731CCD1C261D9F
:1091A000801DD91D321E8A1EE31E3B1F921FEA1F1F
:1091B00041209820EE2044219A21EF214522992236
:1091C000EE2242239623E9233C248F24E2243425F3
:1091D0008525D72528267826C82618276827B72763
:1091E00006285428A228EF283D298929D629222A91
:1091F0006D2AB82A032B4D2B972BE12B2A2C722C8E
:10920000BB2C022D4A2D912DD72D1D2E632EA82E5D
:10921000EC2E302F742FB82FFA2F3D307F30C03016
:10922000013141318131C13100323F327D32BA32B8
:10923000F73234337033AC33E73322345C34953453
:10924000CE3407353F357735AE35E4351A365036EE
:109250008536B936ED36203753378637B737E93795
:10926000193849387938A838D738053932395F394B
:109270008B39B739E2390D3A373A603A893AB23A1E
:10928000DA3A013B283B4E3B733B983BBD3BE03B0E
:10929000043C263C483C6A3C8B3CAB3CCB3CEA3C27
:1092A000093D273D443D613D7D3D993DB43DCE3D69
:1092B000E83D013E1A3E323E493E603E763E8C3EDF
:1092C000A13EB53EC93EDC3EEF3E013F123F233F8B
:1092D000333F433F513F603F6E3F7B3F873F933F6C
:1092E0009E3FA93FB33FBC3FC53FCD3FD53FDC3F8D
:1092F000E23FE83FED3FF13FF53FF93FFB3FFD3FE8
:10930000FF3FFF3FFF3F0000E7382C35002020EFF4
:109310002037202333202620210000800200040073
:10932000080010000002000400080400000200040D
:1093300000080010002000400080040000000080B1
:1093400000000040000000200000001000000008A5
:109350000000000400000002000000010000800086
:109360000000400000002000000010000000080085
:109370000000040000000200000001000080000066
:1093800000080140000C0140000C0140000C0140AD
:10939000000C0140000C0140000C0140000C014099
:1093A0000010014000100140001001400010014079
:1093B0000010014000100140001001400010014069
:1093C0000014014004080140040C0140040C014059
:1093D000040C0140040C0140040C0140040C014049
:1093E000040C01400410014004100140041001402D
:1093F0000410014004100140041001400410014019
:10940000041001400414014008080140080C014008
:10941000080C0140080C0140080C0140080C0140F8
:10942000080C0140080C01400810014008100140E0
:1094300008100140081001400810014008100140C8
:109440000810014008100140081401400C080140B8
:109450000C0C01400C0C01400C0C01400C0C0140A8
:109460000C0C01400C0C01400C0C01400C10014094
:109470000C1001400C1001400C1001400C10014078
:109480000C1001400C1001400C1001400C14014064
:1094900010080140100C0140100C0140100C01405C
:1094A000100C0140100C0140100C0140100C014048
:1094B0001010014010100140101001401010014028
:1094C0001010014010100140101001401010014018
:1094D0001014014000000000000000000000000027
:1094E000000000000000000014080140140C0140BE
:1094F000140C0140140C0140140C0140140C0140E8
:10950000140C0140140C01401410014014100140CF
:1095100014100140141001401410014014100140B7
:109520001410014014100140141401400000000008
:10953000000000000000000000000000000000002B
:10954000FFFFFF0F0FFFFFFFFFF0FFFFFF0FFFFF0A
:10955000FFFFF0FF0FFFFFFFFFF0FFFFFF0FFFFF19
:10956000FFF0FFFF0FFFFFFFFFF0FFFFFF0FFFFF09
:10957000FFFFF0FFFFFF0FFFFFFFFFF0FFFFFF0FF9
:10958000FFF0FFFF0000004040000000000400006A
:109590000040000000000400400000000004000043
:1095A0000040000000040000400000000004000033
:1095B0000040000000000400000040000000000423
:1095C0000000004000040000000000808000000057
:1095D000000800000080000000000800800000007B
:1095E000000800000080000000080000800000006B
:1095F000000800000080000000000800000080005B
:1096000000000008000000800008000000000020AA
:109610002000000000020000002000000000020006
:1096200020000000000200000020000000020000F6
:1096300020000000000200000020000000000200E6
:1096400000002000000000020000002000020000D6
:1096500000000060600000000006000000600000E4
:10966000000006006000000000060000006000002E
:10967000000600006000000000060000006000001E
:10968000000006000000600000000006000000600E
:109690000006000000800200040008001000000224
:1096A000000400080400000200040008001000206C
:1096B0000040008004000000FF7FFFFFFDFFFFFF70
:1096C000FBFFFFFFF7FFFFFFEFFFFFFFFFFDFFFFC8
:1096D000FFFBFFFFFFF7FFFFFBFFFFFFFFFDFFFFAC
:1096E000FFFBFFFFFFF7FFFFFFEFFFFFFFDFFFFFC6
:1096F000FFBFFFFFFF7FFFFFFBFFFFFF0000401FDB
:109700007A1903000000001E897603000000C01CC7
:109710003BDF03000000801BD15704000000401A0B
:109720009FE00400000000199E7B05000000C017A8
:10973000E42C0600000080160DF80600000040151D
:1097400093DE07000000001408E608000000C012C5
:10975000B1110A000000801101650B0000004010EB
:10976000E6E30C000000000F46940E000000C00D60
:10977000467710000000800CB08F12000000400BF4
:10978000D2DE14000000000A5E6317000000C0086B
:10979000601A1A000000800726FC1C00000040062A
:1097A00000002000000000057A1923000000C0031B
:1097B000D5392600000080025851290000004001E0
:1097C000764F2C000000000046252F000000C0FE50
:1097D0002AC63100000080FDA1283400000000FBF3
:1097E0004B1F3800000080F829053B00000000F600
:1097F000EFFE3C0001020304050002030405000122
:109800000304050001020500010203040405000130
:10981000020355050010AA1A55250030AA3A000087
:10982000AA0A55150020AA2A5535FF3F4C98000872
:109830000000002058070000E406000844990008D2
:1098400058070020E0090000EC6600084502040605
:10985000082D0102030404054806070809132D2BEF
:109860001B084104211355152A4006190801A713A6
:109870006F3D1B0895041A8F040125170206040585
:109880000103148020FF8BAA0A0201A415AA0A551D
:109890001500085920AA2A5535FF3F07290301055D
:1098A00004060203127C1573FFFF04FF8080010190
:1098B00029025F6402130A13656A12081201100C70
:1098C0000504060203010103070505280B01020335
:1098D000040206070303040C3D0706040509191FCB
:1098E000191904310506060B14AA1A02312E40FD7F
:1098F0003969260211042F405F020C26405B262A9C
:10990000CD55155515123902017F0316D0071AFFE0
:1099100001013B0261AA0C12080108A8147F993FBB
:109920002340331369720A1608DC91220312100ACD
:1099300017401C12600A16901B014D13796A020031
:04994000080000001B
:020000040800F2
:10FC00004A46545A594D46312D4E3330202020203B
:10FC1000050406020301AA0AAA0AAA0AAA0AAA0A4B
:10FC2000AA0ADE3F00100000FF0131000201664613
:10FC300000400040513800400040004000400101B9
:10FC400000400040FF387B257B257B25FF003333B8
:10FC50000201401F00016626B81E6626FFFFFFFF57
:10FC6000FFFF01010100010000000300000200008D
:04FC70000000AA5591
:04000005080000ED02
:00000001FF
